:020000040000FA
:100000000C94E2010C940A020C940A020C940A0269
:100010000C940A020C940A020C940A020C940A0230
:100020000C940A020C940A020C940A020C940A0220
:100030000C940A020C940A020C940A020C940A0210
:100040000C941D270C940A020C94EB260C94C526E4
:100050000C940A020C940A020C940A020C940A02F0
:100060000C9467270C940A02084AD73B3BCE016EDA
:1000700084BCBFFDC12F3D6C74319ABD56833DDAFF
:100080003D00C77F11BED9E4BB4C3E916BAAAABE0E
:10009000000000803F07634236B79BD8A71A396833
:1000A0005618AEBAAB558C1D3CB7CC5763BD6DED41
:1000B000FD753EF6177231BF000000803F0800005A
:1000C00000BE922449123EABAAAA2ABECDCCCC4C8B
:1000D0003E00000080BEABAAAAAA3E00000000BFFE
:1000E000000000803F0000000000084178D3BB43BF
:1000F00087D1133D190E3CC3BD4282AD2B3E68EC47
:100100008276BED98FE1A93E4C80EFFFBE01C4FFCD
:100110007F3F0000000000004E414E494E495459B7
:10012000494E46CDCCCC3D0AD7233C17B7D13877C2
:10013000CC2B329595E6241FB14F0A0000204100D8
:1001400000C84200401C4620BCBE4CCA1B0E5AAE22
:10015000C59D7400407A10F35A00A0724E18090031
:1001600010A5D4E80000E87648170000E40B54021C
:100170000000CA9A3B000000E1F505000080969857
:1001800000000040420F000000A0860100000010A7
:100190002700000000E803000000006400000000E9
:1001A000000A00000000000100000000002C76D8CA
:1001B00088DC674F0823DFC1DFAE59E1B1B796E5B0
:1001C000E3E453C63AE651997696E8E6C28426EB14
:1001D000898C9B62ED407C6FFCEFBC9C9F40F2BA27
:1001E000A56FA5F490055A2AF75C936B6CF9676DBF
:1001F000C11BFCE0E40D47FEF520E6B500D0ED9014
:100200002E0300943577050080841E080000204EE0
:100210000A000000C80C333333330F986E12831179
:1002200041EF8D2114893BE65516CFFEE6DB18D150
:10023000844B381BF77C1D901DA4BBE42420328422
:10024000725E228100C9F124ECA1E53D274E6F20AA
:10025000445320546865726D6F6D6574657221003A
:10026000543D00495220466C616D65204C657665B1
:100270006C3D00476173206C6576656C3D002349D9
:100280006E76616C6964206B65792100204D756C18
:10029000746973656E736F7273003E482D6669658D
:1002A0006C643A2028004D533D00234E6F20555674
:1002B0002073656E736F722100503D0042543D0003
:1002C0004448543D00234475726174696F6E3D006B
:1002D00054494D45443D0023496E74657276616C06
:1002E0003D0054494D45493D00534156453D004769
:1002F00045540053484F57533D004C6F6767657234
:10030000204E616D653A20004C4F474745520056DC
:10031000455253494F4E00005EBCE2613FDD83C24F
:100320009C7E20A3FD1F41009D23BE46DB65F88C0B
:1003300011AF32CA57E97400000000240027002AD8
:100340000000000000250028002B0023626D7020B3
:100350006661696C6564002357656C636F6D652029
:10036000746F20757365204E616E6F204C6F6767E8
:100370006572005245424F4F5400000000002300B8
:1003800026002900040404040404040402020202F6
:100390000202030303030303010204081020408048
:1003A00001020408102001020408102000000008C7
:1003B000000201000003040700000000000000002C
:1003C00086281E2D11241FBECFEFD8E0DEBFCDBF83
:1003D00012E0A0E0B1E0E8EEF2E702C005900D9275
:1003E000AA37B107D9F725E0AAE7B2E001C01D920C
:1003F000A032B207E1F711E0C1EED1E004C02197CD
:10040000FE010E943037C03ED107C9F70E947E2905
:100410000C9467390C94000090912B0380912A036F
:100420002FEF3FEF981748F4E92FF0E0E65FFC4F1D
:10043000208130E09F5F90932B03C9010895909134
:100440002B0380912A032FEF3FEF981748F4E92FF1
:10045000F0E0E65FFC4F208130E09F5F90932B033C
:10046000C901089591E09093580380937A03109204
:10047000590310927B030895089508950895AF924B
:10048000BF92CF92DF92EF92FF920F931F93CF9381
:10049000DF936C017B018B01040F151FEB015E01E3
:1004A000AE18BF08C017D10759F06991D601ED9178
:1004B000FC910190F081E02DC6010995892B79F717
:1004C000C501DF91CF911F910F91FF90EF90DF90C9
:1004D000CF90BF90AF900895FC0144815581608119
:1004E00071818CE793E00C943F02CF93DF930E94DD
:1004F0006C02EC0142E050E066E571E08CE793E0CD
:100500000E943F028C0F9D1FDF91CF910895FC0147
:10051000538D448D252F30E0842F90E0821B930B68
:10052000541710F0CF96089501970895FC01918D0E
:10053000828D981761F0A28DAE0FBF2FB11D5D9611
:100540008C91928D9F5F9F73928F90E008958FEFB3
:100550009FEF0895FC01918D828D981731F0828D67
:10056000E80FF11D858D90E008958FEF9FEF0895BE
:10057000FC01918D228D892F90E0805C9F4F821B22
:1005800091098F73992708958CE793E00E94B80230
:1005900021E0892B09F420E0822F089580E090E08B
:1005A000892B29F00E94C40281110C940000089547
:1005B000FC01A48DA80FB92FB11DA35ABF4F2C91D8
:1005C000848D90E001968F739927848FA689B789CF
:1005D0002C93A089B1898C91837080648C93938DC6
:1005E000848D981306C00288F389E02D80818F7D69
:1005F00080830895EF92FF920F931F93CF93DF9321
:10060000EC0181E0888F9B8D8C8D98131AC0E8894E
:10061000F989808185FF15C09FB7F894EE89FF891D
:100620006083E889F98980818370806480839FBFBB
:1006300081E090E0DF91CF911F910F91FF90EF90BB
:100640000895F62E0B8D10E00F5F1F4F0F731127CB
:10065000E02E8C8D8E110CC00FB607FCFACFE88906
:10066000F989808185FFF5CFCE010E94D802F1CFB4
:10067000EB8DEC0FFD2FF11DE35AFF4FF0829FB77A
:10068000F8940B8FEA89FB8980818062CFCFCF936A
:10069000DF93EC01888D8823B9F0AA89BB89E889AA
:1006A000F9898C9185FD03C0808186FD0DC00FB650
:1006B00007FCF7CF8C9185FFF2CF808185FFEDCFCE
:1006C000CE010E94D802E9CFDF91CF910895833007
:1006D00081F028F4813099F08230A9F008958730B4
:1006E000A9F08830C9F08430B1F4809180008F7D0A
:1006F00003C0809180008F7780938000089584B537
:100700008F7784BD089584B58F7DFBCF8091B00035
:100710008F778093B00008958091B0008F7DF9CFDE
:10072000CF93DF93EBEBF3E08491E7EAF3E0D4912E
:10073000E3E9F3E0C491CC23A1F081110E946703A7
:10074000EC2FF0E0EE0FFF1FE658FC4FA591B4919F
:10075000EC91ED2381E090E009F480E0DF91CF910E
:10076000089580E090E0FACF1F93CF93DF93282F76
:1007700030E0F901E455FC4F8491F901E856FC4F53
:10078000D491F901EC57FC4FC491CC23A9F0162F5A
:1007900081110E946703EC2FF0E0EE0FFF1FEF5B6B
:1007A000FC4FA591B4918FB7F894EC91111108C04A
:1007B000D095DE23DC938FBFDF91CF911F910895F9
:1007C000DE2BF8CFCF93DF9390E0FC01E856FC4F8F
:1007D00024918C579C4FFC0184918823D1F090E0A8
:1007E000880F991FFC01E95CFC4FA591B491FC01B5
:1007F000EF5BFC4FC591D49161110EC09FB7F89487
:100800008C91E22FE0958E238C932881E223E8835C
:100810009FBFDF91CF9108958FB7F894EC91E22BB1
:10082000EC938FBFF6CF3FB7F8948091F60290918A
:10083000F702A091F802B091F90226B5A89B05C075
:100840002F3F19F00196A11DB11D3FBFBA2FA92F4F
:10085000982F8827BC01CD01620F711D811D911D4C
:1008600042E0660F771F881F991F4A95D1F70895B8
:100870008F929F92AF92BF92CF92DF92EF92FF92B0
:100880006B017C010E9413044B015C01C114D10473
:10089000E104F104B9F00E941304681979098A0986
:1008A0009B09683E73408105910580F321E0C21ADF
:1008B000D108E108F10888EE880E83E0981EA11C9B
:1008C000B11CE4CFFF90EF90DF90CF90BF90AF903E
:1008D0009F908F9008958F929F92AF92BF92EF92C8
:1008E000FF921F93CF93DF93C82F1092140510929D
:1008F000150510921605109217051092180561E063
:100900008FE00E94E20360E08FE00E94B4036C2F4E
:1009100070E090E080E00E94380460E08FE00E9488
:10092000E2038BE990E00197F1F7C0E9D1E00E9482
:100930009003892B71F42197D1F78EEF9FEFDF9110
:10094000CF911F91FF90EF90BF90AF909F908F90AD
:100950000895C0E9D1E00E949003019719F421970E
:10096000D1F7EBCFD8E2C0E810E090E9E92EFF2400
:10097000F3940E949003892B29F481E0E81AF1088E
:10098000C1F7DBCF0E9413044B015C0180E9E82E24
:10099000FF24F3940E949003019729F481E0E81A60
:1009A000F108C1F7CACF0E941304681979098A09AE
:1009B0009B09693271058105910538F0E12FF0E05E
:1009C000E45FFA4F80858C2B8087C69511F41F5FFA
:1009D000C0E8D15051F690E080E0B1CF8F929F9265
:1009E000AF92BF92CF92DF92EF92FF920F931F933D
:1009F000CF93DF938AE0882E912CD0E0C0E0CC2406
:100A0000CA9493E0D92EEE24EA9423E0F22EB12C7E
:100A1000A12C10E000E08091170120E4829FC0012A
:100A20001124816080937C0080917A00806480939F
:100A30007A0080917A0086FDFCCF909178008091B9
:100A400079008927982789270817190790F1A81690
:100A5000B90608F45C018E159F0568F18C159D059B
:100A600008F46C01C80FD91F65E070E080E090E0E9
:100A70000E94380481E0881A910869F60A0D1B1D4E
:100A8000CE01801B910B8C199D098E199F0966E080
:100A900070E00E940837CB01DF91CF911F910F9139
:100AA000FF90EF90DF90CF90BF90AF909F908F908E
:100AB00008958C01D0CF7C01D5CF2FB7F8946091E9
:100AC000F2027091F3028091F4029091F5022FBF2F
:100AD0000895DC0180E0615090F09D919827E92F06
:100AE000EF70F0E0E95EFC4F2491E92FE295EF70A2
:100AF000F0E0E95DFC4FE491822F8E27ECCF089562
:100B0000DC012C911196ED91FC91F8948181822B5E
:100B100081839281322F30959323928387E090E0F6
:100B20000197F1F781818323818383E290E001972C
:100B3000F1F790817894EFECF0E03197F1F79223A0
:100B400081E009F480E00895FC0190810180F28148
:100B5000E02D292F209560FF14C0F8948281822314
:100B600082838181892B8183A3E2B0E01197F1F721
:100B70008281982B9283789487ED90E00197F1F72A
:100B80000895F8948281822382838181892B8183D5
:100B9000AFEFB0E01197F1F78281982B92837894B0
:100BA0008FE090E0EBCFDF92EF92FF920F931F93D5
:100BB000CF93DF93EC01D62EE42E08E010E0FF2463
:100BC000F39461E08D2D8F2109F460E0CE010E9445
:100BD000A405FF0C01501109A1F7E11010C0F89411
:100BE000E981FA8191818881809589238183E981D6
:100BF000FA81928188818095892382837894DF911C
:100C0000CF911F910F91FF90EF90DF900895EF9299
:100C1000FF920F931F93CF93DF938C017B0140E0F2
:100C200065E50E94D305E70188E0E80EF11C6991B3
:100C300040E0C8010E94D305CE15DF05C1F7DF9162
:100C4000CF911F910F91FF90EF900895FC0190813B
:100C50000180F281E02DF8948181292F2095822353
:100C6000818378943DE743E050E0315029F1DA0187
:100C70001197F1F780818923C1F3F894828182234F
:100C800082838181892B81837894ABE7B7E01197C8
:100C9000F1F7F894818182238183A3E1B1E0119778
:100CA000F1F78081982381E009F080E07894E3E611
:100CB000F6E03197F1F7089580E008956F927F9202
:100CC0008F929F92AF92BF92CF92DF92EF92FF925C
:100CD0000F931F93CF93DF93EC017B018A018E81E9
:100CE0009F810E942606811102C090E037C0B701A3
:100CF0008E819F810E94070640E06EEB8E819F816E
:100D00000E94D3057801680189E0C80ED11CAE802D
:100D1000BF8088E0882E912C712C66246394C501D5
:100D20000E94800581117628660CE1E08E1A9108F8
:100D3000B1F7F70171927F01EC15FD0541F78E8146
:100D40009F810E942606813081F668E0C8010E94DA
:100D5000690591E0F80120852813C7CF892FDF911D
:100D6000CF911F910F91FF90EF90DF90CF90BF90A8
:100D7000AF909F908F907F906F900895CF93DF9367
:100D8000CDB7DEB729970FB6F894DEBF0FBECDBF43
:100D9000AE014F5F5F4F0E945E06882331F08D8168
:100DA0008F33A9F020F48F31A1F080E007C08F3598
:100DB00021F08F37D1F78CE001C08BE029960FB678
:100DC000F894DEBF0FBECDBFDF91CF9108958AE0CA
:100DD000F5CF89E0F3CF089580912A0390912B03FA
:100DE000891B990B089508952091CE02260F332771
:100DF000331F21323105ECF420915203FC0190E0C5
:100E000080E0243069F082E00895A091CE02219123
:100E1000AC0142555D4FA40FB52FB11D2C93019627
:100E2000861798F38091CE02680F6093CE0280E01F
:100E3000089581E008951092520381E08093510358
:100E400010922C0361E082E10E94B40361E083E12F
:100E50000E94B403E9EBF0E080818E7F8083808183
:100E60008D7F808388E48093B80085E48093BC0004
:100E7000089510922B0310922A0310925903109296
:100E80007B030E941B078CE392E0909309038093FD
:100E900008038DE392E0909307038093060308957F
:100EA000CF93DF9391E09093AD028823B9F0C09186
:100EB000B800D091BA008091BC008A7B8093BC00BE
:100EC00060E082E10E94B40360E083E10E94B40329
:100ED0000E941B07D093BA00C093B800DF91CF9156
:100EE0000895CF92DF92EF92FF920F931F93CF93CB
:100EF000DF93D0917B0381E0D13208F09CC0C09198
:100F00007A030E9413046B017C01809152038111CA
:100F10006CC082E08093520381E0809351038FEF95
:100F20008093500310924F03D0934E03AAE5B3E091
:100F3000EEE2F3E080E0D8138DC010922D03809193
:100F40002D03CC0FC82BC0932D0380912C0381302F
:100F500009F084C010922C030E9413046B017C01E1
:100F600080912D038093BB00809154039091550391
:100F7000A0915603B0915703892B8A2B8B2BA1F09C
:100F80000E941304009154031091550320915603BD
:100F9000309157036C197D098E099F0906171707B1
:100FA0002807390708F442C08091BC0083FDD8CFE0
:100FB00085EC8093BC000E9413046B017C0180913E
:100FC0005203823009F44CC0809150038F3F09F4E2
:100FD00069C080915003803209F466C0809150034B
:100FE000803309F463C084E026C08091540390915B
:100FF0005503A0915603B0915703892B8A2B8B2B55
:1010000009F483CF0E9413040091540310915503F7
:1010100020915603309157036C197D098E099F0961
:10102000061717072807390708F06FCF8091530379
:101030000E94500785E01092590310927B03109292
:101040005803DF91CF911F910F91FF90EF90DF90A8
:10105000CF9008959D9191938F5F6DCF85EEA9CF2D
:101060008091540390915503A0915603B09157037A
:10107000892B8A2B8B2B09F4A2CF0E941304009199
:1010800054031091550320915603309157036C1966
:101090007D098E099F09061717072807390708F0E9
:1010A0008ECFC4CF80E0C7CF82E0C5CF83E0C3CF6F
:1010B000CF92DF92EF92FF920F931F93CF93DF9324
:1010C000D82FC62F613208F098C00E9413046B011C
:1010D0007C018091520381116BC081E080935203A7
:1010E000809351039FEF9093500310924F039C0FF6
:1010F00090934E0380932D0380912D03DD0FD82B09
:10110000D0932D0380912C03813009F078C0109288
:101110002C030E9413046B017C0180912D038093AA
:10112000BB008091540390915503A0915603B09158
:101130005703892B8A2B8B2BA1F00E94130400915B
:1011400054031091550320915603309157036C19A5
:101150007D098E099F09061717072807390708F424
:1011600048C08091BC0083FDD8CF85EC8093BC0043
:101170000E9413046B017C0180915203813009F4B9
:1011800040C080914F038C1710F4C0914F03EEE2E2
:10119000F3E0AAE0B3E080E08C1355C08C2FDF9120
:1011A000CF911F910F91FF90EF90DF90CF90089516
:1011B0008091540390915503A0915603B091570329
:1011C000892B8A2B8B2B09F484CF0E941304009166
:1011D00054031091550320915603309157036C1915
:1011E0007D098E099F09061717072807390708F098
:1011F00070CF809153030E945007C0E0CFCF85EE9F
:10120000B5CF8091540390915503A0915603B091AE
:101210005703892B8A2B8B2B09F4AECF0E94130422
:1012200000915403109155032091560330915703B8
:101230006C197D098E099F090617170728073907BA
:1012400008F09ACFD6CF91919D938F5FA5CF089547
:10125000E0912B0380912A03E81730F4F0E0E65F79
:10126000FC4F808190E008958FEF9FEF0895CF921B
:10127000DF92EF92FF920F931F93CF93DF937C0146
:10128000CB018A0120915803222389F0EB016B01E5
:10129000C40ED51ECC15DD0569F06991D701ED911D
:1012A000FC910190F081E02DC7010995F3CF642FE7
:1012B0000E94F406C801DF91CF911F910F91FF901A
:1012C000EF90DF90CF900895CF93DF931F92CDB72B
:1012D000DEB76983209158032223F9F020917B0324
:1012E000203258F021E030E0FC013383228390E08B
:1012F00080E00F90DF91CF91089580915903E82FFE
:10130000F0E0E65AFC4F998190838F5F80935903F8
:1013100080937B0381E090E0ECCF61E0CE01019609
:101320000E94F406F7CFCF93C82F83E50E943202C4
:101330006DE289E194E00E9464096C2F89E194E0F8
:101340000E946409CF910C94710790E080E00895A9
:10135000FC0124813581232B41F00E946C0269E15C
:1013600070E080E090E00C94380408950E945808E2
:1013700010922B0380932A030895CF93C82F87E7F9
:101380000E9432026C2F89E194E00E9464090E945D
:10139000710787E70E94320261E070E087E790E022
:1013A0000E94B6090E941F02C82F0E9471078C2F4D
:1013B000CF910895CF93DF93C82F87E70E94320221
:1013C0006C2F89E194E00E9464090E94710787E70D
:1013D0000E94320262E070E087E790E00E94B60966
:1013E0000E941F02D82F80E0C82F0E941F02C82B26
:1013F000D92B0E947107CE01DF91CF91089587E725
:101400000E94320264EF89E194E00E9464096EE276
:1014100089E194E00E9464090E94710765E070E030
:1014200080E090E00E94380486EF0C94DA094F9235
:101430005F926F927F928F929F92AF92BF92CF9264
:10144000DF92EF92FF92CF93DF9300D000D01F92F4
:10145000CDB7DEB70E94FF094C01B12CA12C209121
:10146000E1042295220F220F207C2C5C298387E740
:101470000E94320264EF89E194E00E94640969816C
:1014800089E194E00E9464090E9471078091E1045F
:10149000811174C165E070E080E090E00E94380442
:1014A00086EF0E94DA09B0E0A0E0CC24D82EE92E25
:1014B000FA2E88EF0E94BD09A7019601282B2983E7
:1014C0003A834B835C833091E1043D838091F60441
:1014D0009091F704A5019401281B390B410951098A
:1014E000A091F404B091F5040E9416334B015C0105
:1014F000AFE0B594A79497948794AA95D1F760919B
:10150000EE047091EF04072E000C880B990BBBE0E2
:10151000660F771F881F991FBA95D1F72091F004A5
:101520003091F104032E000C440B550B280D391D8E
:101530004A1D5B1D0E94F732820E931EA41EB51E2B
:101540007501640140EAC41A4FE0D40AE108F108C9
:10155000A7019601C701B6010E94F8364B015C0154
:101560008CE0B594A794979487948A95D1F7A0912D
:10157000E604B091E7040E9421332B013C019DE079
:1015800075946794579447949A95D1F7A091E8047D
:10159000B091E904A50194010E9421339C015527D3
:1015A00037FD5095452F240D351D461D571D2E5FC7
:1015B0003F4F4F4F5F4F62E05595479537952795C1
:1015C0006A95D1F730584F4F5F4FA091F204B09118
:1015D000F3040E9416332B013C017FE0769467945C
:1015E000579447947A95D1F788E090E05D81851B08
:1015F000910929813A814B815C8104C056954795B8
:10160000379527958A95D2F729833A834B835C8354
:10161000A091EA04B091EB04A50194010E9421334A
:101620004B015C01EBE0B594A79497948794EA95FD
:10163000D1F7A091E404B091E504A70196010E94BE
:101640002133FBE09595879577956795FA95D1F7C6
:10165000680D791D8A1D9B1D8090E2049090E30423
:10166000092C000CAA08BB08A2E0880C991CAA1C33
:10167000BB1CAA95D1F7680D791D8A1D9B1D0D8095
:1016800004C0660F771F881F991F0A94D2F76E5FF8
:101690007F4F8F4F9F4F24E030E040E050E00E94AA
:1016A000F73289819A81AB81BC81821B930BA40B99
:1016B000B50B9C01AD0160E573EC80E090E00D801E
:1016C00004C096958795779567950A94D2F70E94FE
:1016D000F83697FD66C0660F771F881F991FA30114
:1016E00092010E94603369017A019927F7FC9A956B
:1016F0008F2D7E2D6D2D9B01AC010E94F8369B0134
:10170000AC01AEEDBBE00E9416334B015C01A3E4DB
:10171000B3EEA70196010E942433BC01992777FDFF
:101720009095892F4501BB2497FCB094AB2C680D94
:10173000791D8A1D9B1D6153714F8F4F9F4F44E050
:1017400095958795779567954A95D1F76C0D7D1D91
:101750008E1D9F1D0F900F900F900F900F90DF9197
:10176000CF91FF90EF90DF90CF90BF90AF909F9080
:101770008F907F906F905F904F900895813029F403
:1017800068E070E080E090E089CE823029F46EE07D
:1017900070E080E090E082CE6AE170E080E090E06E
:1017A0007DCEA30192010E94603369017A01CC0CC5
:1017B000DD1CEE1CFF1C99CFBF92CF92DF92EF92FF
:1017C000FF920F931F93CF93DF93EC01B62EC72E9A
:1017D0008D85811105C0CE010E94260681110EC0A3
:1017E0001B861D861C8680E0DF91CF911F910F9193
:1017F000FF90EF90DF90CF90BF90089540E060EFB2
:10180000CE010E94D30501E0E12CD12C11E0CE01E4
:101810000E948005F82ECE010E94800591E0F91209
:1018200018C0813099F51134D8F2DB86D11002C08E
:1018300081E08D878B81882399F22396EB2DFC2DF7
:10184000CF01089629912193E817F907D9F781E08C
:10185000CBCFEE2DF0E0F8120FC08B851817A0F457
:10186000DE01AE0FBF1F13968C91802379F4F12C0B
:10187000193008F41C87D12EEC0FFD1F8381902FA7
:101880009095892383830AC08113F1CFFE01EE0D69
:10189000F11D8381802B8383FF24F3946F2DCE0170
:1018A0000E94A4051F5F000F11F4E39401E087E09C
:1018B0008E1508F0ACCFB7CFDF92EF92FF920F9367
:1018C0001F93CF93DF937C018B01D42EDC011696FE
:1018D000ED91FC911386158614861286118610866A
:1018E00017821682158214821382C0E0B801F701B4
:1018F000868197810E94DC0BD82F882329F0DC1683
:1019000029F0CF5FDC1690F7D0E009C067E0C8018E
:101910000E946905D80117969C918913F2CF8D2FEB
:10192000DF91CF911F910F91FF90EF90DF9008957D
:101930000F931F93CF93DF93FC0104811581011551
:10194000110539F4FB011082DF91CF911F910F91A6
:101950000895415051094017510708F48A01EB01DD
:10196000FC0160817181A801CE010E943E39C00F47
:10197000D11F1882E9CFCF93DF93C091BC04D091DF
:10198000BD04209761F08991882349F0082E000C4E
:10199000990B0E941839FE0131978083F4CFDF91B3
:1019A000CF910895FC0180819181009711F00C94F2
:1019B000602D60E070E0CB010895AF92BF92CF92AE
:1019C000DF92EF92FF920F931F93CF93DF93DC018F
:1019D000CD90DC901197C114D10439F01496CD91BB
:1019E000DC918C017601209761F4DF91CF911F91FA
:1019F0000F91FF90EF90DF90CF90BF90AF90089540
:101A000075015701BFEFAB1ABB0AF7018081082EA1
:101A1000000C990B0E948931892B91F72197CC0DED
:101A2000DD1D8881082E000C990B0E948931892BBD
:101A300029F0CE15DF0510F02197F3CFAE014F5FEF
:101A40005F4F4E195F09D80115965C934E9314971A
:101A5000CE14DF0420F4B701C6010E942039D8015A
:101A6000ED91FC91119714968D919C91E80FF91FBF
:101A70001082BBCFFB0144815581FC01248135815B
:101A80002417350778F080819181009759F0FB0188
:101A9000608171816115710529F00E94303921E062
:101AA000892B09F020E0822F08950F931F93CF9385
:101AB000DF938C01EB01FC01808191810097E1F0C3
:101AC0006881798161157105A9F0428153812C816A
:101AD0003D814217530770F00E9429398C819D8106
:101AE000F801958384831D821C82DF91CF911F9121
:101AF0000F9108950E94D23788819981F8019183CE
:101B000080838A819B81938382838C819D8195834D
:101B10008483198218821B821A82E5CFCF93DF93C8
:101B2000EC0188819981009711F00E94D2371982C7
:101B300018821D821C821B821A82DF91CF91089528
:101B4000FC0180819181009711F00C94D2370895A7
:101B50000C94D2370F931F93CF93DF93EC018881BE
:101B60009981009759F02A813B812617370730F079
:101B700081E0DF91CF911F910F9108958B016F5FED
:101B80007F4F0E945B38009759F0998388831B83AD
:101B90000A832C813D81232B59F7FC011082E8CF69
:101BA00080E0E7CFEF92FF920F931F93CF93DF93E5
:101BB0006115710541F480E0DF91CF911F910F9184
:101BC000FF90EF90089541155105B1F07B01EC01B4
:101BD0000C811D81040F151FB8010E94AA0D8823D6
:101BE00051F3288139818C819D81B701820F931F28
:101BF0000E9429391D830C8381E0DECF0F931F9350
:101C0000CF93DF9300D0CDB7DEB78C0119821A8253
:101C100041E050E0BE016F5F7F4F0E94D20D811105
:101C200003C0C8010E948E0DC8010F900F90DF9174
:101C3000CF911F910F910895CF93DF93EC01FB019A
:101C400001900020E9F73197AF01461B570B0E9426
:101C5000D20D811103C0CE010E948E0DCE01DF9105
:101C6000CF910895CF93DF93EC01FB01448155811F
:101C7000608171810E94D20D811103C0CE010E944A
:101C80008E0DCE01DF91CF910895FB0101900020D0
:101C9000E9F73197AF01461B570B0C94D20DFB01AE
:101CA00044815581608171810C94D20DEF92FF9235
:101CB0000F931F93CF93DF93EC018B01CB010E9415
:101CC0008E2D7C01BC01CE010E94AA0D81110BC09A
:101CD000CE010E948E0DCE01DF91CF911F910F9109
:101CE000FF90EF900895FD82EC82B8018881998180
:101CF0000E94872DF0CFFC01118210821382128284
:101D0000158214820C94560EEF92FF920F931F933C
:101D1000CF93DF93EC017B018A01BA010E94AA0DE7
:101D200081110BC0CE010E948E0DCE01DF91CF91AB
:101D30001F910F91FF90EF9008951D830C83B701C1
:101D4000888199810E942939F0CFFB010190002000
:101D5000E9F73197AF01461B570B0C94840E0F9394
:101D60001F93CF93DF93CDB7DEB762970FB6F8948A
:101D7000DEBF0FBECDBF8C01CB01F80111821082F6
:101D800013821282158214824AE0BE016F5F7F4F78
:101D90000E94972DBE016F5F7F4FC8010E94A50E64
:101DA00062960FB6F894DEBF0FBECDBFDF91CF9124
:101DB0001F910F910895CF93DF93EC01FB018617DC
:101DC000970749F0608171816115710541F0448187
:101DD00055810E94840ECE01DF91CF9108950E941B
:101DE0008E0DF9CFFC0111821082138212821582AE
:101DF00014820C94DB0EFC01118210821382128279
:101E000015821482FB0101900020E9F73197AF01A0
:101E1000461B570B0C94840EAF92BF92CF92DF9269
:101E2000EF92FF920F931F93CF93DF936C015B01AF
:101E30007A0189012417350720F48F2D7901042FA9
:101E4000182F68E571E0C6010E94FB0ED5011496BB
:101E5000CD91DC91EC16FD06E0F40C171D0708F49B
:101E6000E801D501ED91FC911197EC0FFD1F108158
:101E700010826D917C916E0D7F1DC60161157105FB
:101E8000A1F00E94A50EF50180819181C80FD91F94
:101E90001883C601DF91CF911F910F91FF90EF90B2
:101EA000DF90CF90BF90AF9008950E948E0DEBCF42
:101EB000CF93DF93EC01FB01248135810E940C0F4D
:101EC000CE01DF91CF9108950F931F93CF93DF93AE
:101ED000CDB7DEB72C970FB6F894DEBF0FBECDBFDF
:101EE000FC01248135811216130664F48C0125311E
:101EF00031059CF40E94750264E170E080E090E09E
:101F00000E9438042C960FB6F894DEBF0FBECDBFEA
:101F1000DF91CF911F910F9108952FE030E050E0B5
:101F200040E0BC01CE0107960E940C0FCE0107963F
:101F30000E946C0269E170E080E090E00E94380449
:101F40004FE050E0B801CE0101960E94580FBE014B
:101F50006F5F7F4FCE0107960E94550DCE0101960F
:101F60000E94A00DCE0107960E94750264E170E008
:101F700080E090E00E94380468E571E0CE010796A9
:101F80000E94A50ECE0107960E94A00DBBCFEF9236
:101F9000FF920F931F93CF93DF93CDB7DEB7A19737
:101FA0000FB6F894DEBF0FBECDBF7C01CB01BA01E6
:101FB000F70111821082138212821582148242E08C
:101FC000420F8E010F5F1F4F0E943E2D009789F038
:101FD000BC01C7010E94A50EA1960FB6F894DEBF02
:101FE0000FBECDBFDF91CF911F910F91FF90EF906A
:101FF0000895C7010E948E0DEFCF0F931F93CF93CB
:10200000DF938C01EB0188E2FB0111928A95E9F7DD
:102010004BE050E069E571E0CE010E943E391B863D
:1020200081E090E0A0E0B0E08C879D87AE87BF871D
:10203000F80185899689A789B08D888B998BAA8BA1
:10204000BB8B82E090E0A0E0B0E08C8B9D8BAE8BF0
:10205000BF8B1CA21DA21EA21FA280E090E0A8E4DC
:10206000B4E4888F998FAA8FBB8F80E090E0A8E4BA
:10207000B4EC8C8F9D8FAE8FBF8F8DEC9CECACE45D
:10208000BEE388A399A3AAA3BBA3DF91CF911F911D
:102090000F910895AF92BF92CF92DF92EF92FF928D
:1020A0000F931F93CF93DF938C01EB0184E2FB012D
:1020B00011928A95E9F78EE10E94320263E089E18C
:1020C00094E00E9464090E94710766E08EE10E941C
:1020D000580810922B0380932A038630F0F30E9455
:1020E0001F02A82E0E941F02B82E0E941F02E82E77
:1020F0000E941F02F82E0E941F02C82E0E941F027B
:10210000D82E60E07A2D6B29072E000C880B990BD6
:102110000E94C131F801658376838783908760E0F0
:102120007C2D6D29072E000C880B990B0E94C13164
:10213000F801618772878387948760E07E2D6F291D
:10214000072E000C880B990B0E94C131F80165879E
:1021500076878787908B118A128A138A148A84E281
:1021600090E0A0E0B0E088839983AA83BB8385894F
:102170009689A789B08D8C839D83AE83BF8382E0CF
:1021800090E0A0E0B0E088879987AA87BB87188A8B
:10219000198A1A8A1B8AC0900A01D0900B01E0901C
:1021A0000C01F0900D01A701960165817681878170
:1021B00090850E94703420E030E048EC52E40E94A8
:1021C00020326C8B7D8B8E8B9F8BA7019601F80143
:1021D00061857285838594850E94703420E030E0AB
:1021E00048EC52E40E942032688F798F8A8F9B8F4F
:1021F0002091060130910701409108015091090199
:10220000F80165857685878590890E94703420E085
:1022100030E048EC52E40E9420326C8F7D8F8E8F2C
:102220009F8F81E0DF91CF911F910F91FF90EF90F1
:10223000DF90CF90BF90AF90089585ED8093BC0064
:102240008091540390915503A0915603B091570388
:102250000796A11DB11D23E0B695A7959795879583
:102260002A95D1F72091BC0024FD03C0109252039F
:102270000895409154035091550360915603709115
:102280005703452B462B472B69F30097A105B10552
:1022900041F025E32A95F1F700000197A109B10962
:1022A000E1CF809153030C9450074F925F926F924D
:1022B0007F928F929F92AF92BF92CF92DF92EF92D6
:1022C000FF92CF93DF93CDB7DEB7CA54D1090FB6D3
:1022D000F894DEBF0FBECDBF68E571E0CE01C796B2
:1022E0000E94FB0E68E571E0CE01CD960E94FB0EC8
:1022F000BE016F5F7F4F88EC94E00E944A10CD884A
:10230000DE88EF88F88C20E030E040E251E4C7013D
:10231000B6010E9420322B013C01898D9A8DAB8D34
:10232000BC8D2B968CAF9DAFAEAFBFAF2B9720E08F
:1023300030E040E251E4BC01CD010E9420324B016B
:102340005C0120E030E040E251E46D8D7E8D8F8DA8
:1023500098A10E94203227966CAF7DAF8EAF9FAFC1
:102360002797C701B60190582B962CAD3DAD4EADC9
:102370005FAD2B970E9411342BED3FE049EC5FE3FA
:102380000E949233209135043091360440913704F5
:10239000509138040E9492336B017C0120E030E0C0
:1023A000A9010E94BA3187FF0AC02BED3FE049EC3A
:1023B00050E4C701B6010E9492336B017C012BED02
:1023C0003FE049EC50E4C701B6010E943F351816C2
:1023D00054F42BED3FE049EC50E4C701B6010E94F4
:1023E00091336B017C0120E030E044E353E4C7010A
:1023F000B6010E9420322BED3FE049E450E40E94F8
:1024000070346B017C0120E0BC01A601CE018B96EB
:102410000E94C70F61E671E0CE0185960E94FB0E17
:10242000BE01655D7F4FCE0185960E94320E6BE640
:1024300071E00E941C0EBC0182EC94E00E94DB0E55
:10244000CE0185960E94A00DCE018B960E94A00D14
:1024500020E030E044EB52E4C701B6010E94BA31FB
:1024600018160CF4BFC120E030E040E05FE3C70184
:10247000B6010E949233AB01BC0120E0CE018B96E5
:102480000E94C70F62E771E0CE0185960E94FB0EA5
:10249000BE01655D7F4FCE0185960E94320EBC0164
:1024A000CE01C7960E94DB0ECE0185960E94A00D3C
:1024B000CE018B960E94A00D65E771E0CE01CD960E
:1024C0000E94A50E60E771E0CE0185960E94FB0E8A
:1024D000BE01635C7F4FCE0185960E94320EBC0127
:1024E000CE01C7960E944F0ECE0185960E94A00D88
:1024F0000E945D05C0907A02D0907B02E0907C0241
:10250000F0907D026C197D098E099F090E94BF31F0
:1025100020E030E04AE754E40E947034AB01BC0193
:1025200023E0CE018B960E94C70F65E871E0CE01D3
:1025300085960E94FB0EBE01655D7F4FCE0185969C
:102540000E94320E6CE771E00E941C0EBC0184EA0E
:1025500094E00E94DB0ECE0185960E94A00DCE0174
:102560008B960E94A00D64EA74E0CE0185960E94CD
:10257000F20ECE0185960E94A809CE0185960E9492
:10258000A00D62EC74E0CE0185960E94F20ECE01A1
:1025900085960E94A809CE0185960E94A00DBE01D5
:1025A000695C7F4FCE0185960E94F20ECE01859622
:1025B0000E94640FCE0185960E94A00D64EA74E02B
:1025C000CE0185960E94F20E62EC74E0CE018596F3
:1025D0000E94320EBE01695C7F4F0E94320EBC0128
:1025E000CE01C7960E94DB0ECE0185960E94A00DFB
:1025F0006AE972E0CE0185960E947B0ECE01859637
:102600000E94A809CE0185960E94A00D68E571E0A0
:1026100082EC94E00E94A50E21E0B301A201CE015C
:1026200085960E94C70FBE016B5D7F4F82EC94E0E0
:102630000E944F0ECE0185960E94A00D21E02796A4
:102640004CAD5DAD6EAD7FAD2797CE01C1960E94BA
:10265000C70F21E0B501A401CE018B960E94C70FE0
:1026600060E771E0CE0185960E94FB0EBE01655DBC
:102670007F4FCE0185960E94320E60E771E00E9486
:102680001C0EBE016F5C7F4F0E94320E6FE771E03F
:102690000E941C0EBC0182EC94E00E944F0ECE0101
:1026A00085960E94A00DCE018B960E94A00DCE01B2
:1026B000C1960E94A00D62EC74E0CE0185960E9446
:1026C000F20ECE0185960E94A809CE0185960E9441
:1026D000A00DA3019201C301B2010E9420326B013F
:1026E0007C01A5019401C501B4010E9420329B0127
:1026F000AC01C701B6010E9492336B017C012796A1
:102700002CAD3DAD4EAD5FAD2797CA01B9010E941A
:1027100020329B01AC01C701B6010E9492330E9496
:10272000A2356B017C0163E871E082EC94E00E94C9
:10273000A50E21E0B701A601CE0185960E94C70F24
:10274000BE016B5D7F4FCE018B960E94F20E60E85A
:1027500071E0CE018B960E941C0EBC0182EC94E0CD
:102760000E944F0ECE018B960E94A00DCE01859641
:102770000E94A00D62EC74E0CE0185960E94F20EDC
:10278000CE0185960E94640FCE0185960E94A00D11
:1027900068E571E082EC94E00E94A50E65E070E0CF
:1027A00080E090E00E943804CE01CD960E94A00DFA
:1027B000CE01C7960E94A00DC65BDF4F0FB6F894FE
:1027C000DEBF0FBECDBFDF91CF91FF90EF90DF90C6
:1027D000CF90BF90AF909F908F907F906F905F90C1
:1027E0004F90089520E030E044E353E4C701B60180
:1027F0000E94BA31181694F0A701960160E070E8C3
:1028000084E393E40E949133AB01BC0120E0CE014C
:102810008B960E94C70F67E771E036CE20E030E06C
:1028200047E853E4C701B6010E94BA31181694F183
:1028300020E030E044E353E4C701B6010E94913345
:1028400020E030E040E05FE30E949233AB01BC0146
:1028500020E0CE018B960E94C70F67E771E0CE01A2
:1028600085960E94FB0EBE01655D7F4FCE01859669
:102870000E94320EBC01CE01C7960E94DB0ECE0133
:1028800085960E94A00DCE018B960E94A00D6AE74E
:1028900071E014CEA701960160E070E084EB93E450
:1028A0000E94913320E030E040E05FE30E949233E9
:1028B0000E94E234CE018B960E94AF0E62E771E077
:1028C000CECFFF920F931F93CF93DF93EC01F62EA1
:1028D00008811981C8010E94E132F81621F06F2D9C
:1028E000C8010E94E932CE01DF91CF911F910F9173
:1028F000FF900895EF92FF920F931F93CF93DF9372
:1029000000D0CDB7DEB705E214E0855294407C01DB
:10291000C701800F911F9A838983F80161918F010C
:10292000CE0101960E946114F4E001371F0781F780
:1029300085E294E00F900F90DF91CF911F910F915E
:10294000FF90EF900895EF92FF920F931F93CF9314
:10295000DF9300D0CDB7DEB701E714E08157944094
:102960007C01C701800F911F9A838983F8016191CF
:102970008F01CE0101960E946114F4E008391F070F
:1029800081F781E794E00F900F90DF91CF911F9135
:102990000F91FF90EF9008954F925F926F927F9208
:1029A0008F929F92AF92BF92CF92DF92EF92FF925F
:1029B0000F931F93CF93DF93CDB7DEB76E970FB60C
:1029C000F894DEBF0FBECDBF6FE073E0CE0101967D
:1029D0000E947B0EBE016F5F7F4F8CEB94E00E94E4
:1029E0003A0D182FCE0101960E94A00D112399F1E6
:1029F00067E871E0CE0101960E94FB0E68E974E081
:102A0000CE0101960E94320EBC0182EC94E00E943D
:102A1000DB0ECE0101960E94A00D61E971E0CE01AE
:102A200007960E94FB0E62EC74E0CE0107960E94AE
:102A3000320EBC01CE0101960E94F20ECE0101962B
:102A40000E94640FCE0101960E94A00DCE01079650
:102A50000E94A00D52C068E073E0CE0101960E9472
:102A60007B0EBE016F5F7F4F8CEB94E00E943A0DAE
:102A7000182FCE0101960E94A00D112369F06AEF74
:102A800072E082EC94E00E94560E6EE974E082ECF3
:102A900094E00E944F0EC1CF63EF72E0CE01019629
:102AA0000E947B0EBE016F5F7F4F8CEB94E00E9413
:102AB0003A0D182FCE0101960E94A00D1123C9F1E5
:102AC00027E030E046E050E060EB74E0CE01019694
:102AD0000E940C0FBE016F5F7F4F8AEA94E00E9454
:102AE000550DCE0101960E94A00D8AEA94E00E9445
:102AF000D20C672B21F41092FC0281E003C081E02C
:102B00008093FC026E960FB6F894DEBF0FBECDBF69
:102B1000DF91CF911F910F91FF90EF90DF90CF90B9
:102B2000BF90AF909F908F907F906F905F904F90ED
:102B300008956FEE72E0CE0101960E947B0EBE01F9
:102B40006F5F7F4F8CEB94E00E943A0D182FCE01FF
:102B500001960E94A00D112309F4B8C08091AB0228
:102B60009091AC021816190644F688EC90E0909308
:102B70000501809304018CE793E00E9447031D86C2
:102B80001E861F86188ACC24C394D12C60EC462E56
:102B900063E0562E5E012DE0A20EB11C3E0131E134
:102BA000630E711C8091AB029091AC028C159D0557
:102BB0000CF4A3CF8091040190910501813C9340D6
:102BC00024F05092050140920401009104011091FB
:102BD0000501750148018A189B08C4018E0D9F1DCF
:102BE0000E94E132F70181937F01E615F705A9F70D
:102BF000C8010496909305018093040147E8E42EF0
:102C000042E0F42E03581240C8018E0D9F1D0E9411
:102C1000E132F70181937F01FBEAEF16F2E0FF0654
:102C200099F74D855E856F85788923E0CE010796FB
:102C30000E94C70FBE01695F7F4FCE0101960E94BF
:102C4000F20E6CE771E0CE0101960E941C0EBC01F1
:102C500082EC94E00E94DB0ECE0101960E94A00D52
:102C6000CE0107960E94A00D67E872E0CE010196A2
:102C70000E94FB0EBE016F5F7F4F82EC94E00E94CA
:102C80004F0ECE0101960E94A00D62EC74E0CE01C1
:102C900001960E94F20ECE0101960E94640FCE01B1
:102CA00001960E94A00D80910401909105018496E7
:102CB000909305018093040164E170E080E090E06E
:102CC0000E9438042FEFC21AD20A6CCF69EE72E06C
:102CD000CE0101960E947B0EBE016F5F7F4F8CEB91
:102CE00094E00E943A0D182FCE0101960E94A00D8B
:102CF0001123F1F126E030E045E050E060EB74E0B4
:102D0000CE0101960E940C0FBE016F5F7F4F8AEAD1
:102D100094E00E94550DCE0101960E94A00D8AEA12
:102D200094E00E94D20C672B19F410928602E5CE33
:102D300081E08093860288EC90E090930501809377
:102D400004011092AC021092AB0210928202109217
:102D5000830210928402109285020E945D056093A6
:102D60007E0270937F028093800290938102C5CE91
:102D700062EE72E0CE0101960E947B0EBE016F5F93
:102D80007F4F8CEB94E00E943A0D182FCE010196F4
:102D90000E94A00D112309F47FC08091B40490918A
:102DA000B504079708F4A9CE46E050E060EB74E064
:102DB000CE0101960E94580FBE016F5F7F4F8AEAD5
:102DC00094E00E94550DCE0101960E94A00D8091C5
:102DD000AA049091AB04009709F45AC00E945C2D9C
:102DE0006093130170931401809315019093160161
:102DF00067ED72E082EC94E00E94560E4091130160
:102E000050911401609115017091160122E0CE01DC
:102E100007960E94C70FBE01695F7F4FCE010196E2
:102E20000E94F20E63E971E0CE0101960E941C0E31
:102E3000BC0182EC94E00E944F0ECE0101960E94EC
:102E4000A00DCE0107960E94A00D62EC74E0CE01A9
:102E500001960E94F20ECE0101960E94640FCE01EF
:102E600001960E94A00D0E945D0528EE33E040E02F
:102E700050E00E946033CA01B9010E94BF316093E3
:102E8000010370930203809303039093040335CEF0
:102E900060E070E0CB01A4CF60ED72E0CE0101965E
:102EA0000E947B0EBE016F5F7F4F8CEB94E00E940F
:102EB0003A0D182FCE0101960E94A00D112309F49E
:102EC0006BC08091B4049091B504079708F415CEB7
:102ED00046E050E060EB74E0CE0101960E94580F8E
:102EE000BE016F5F7F4F8AEA94E00E94550DCE01CC
:102EF00001960E94A00D8091AA049091AB040097C6
:102F000009F446C00E945C2D60930001709301019A
:102F1000809302019093030165EC72E082EC94E0EF
:102F20000E94560E409100015091010160910201F2
:102F30007091030121E0CE0107960E94C70FBE01E8
:102F4000695F7F4FCE0101960E94F20E63E971E046
:102F5000CE0101960E941C0EBC0182EC94E00E94FE
:102F60004F0ECE0101960E94A00DCE0107960E9441
:102F7000A00D62EC74E0CE0101960E94F20ECE012B
:102F800001960E94640FCE0101960E94A00DB5CD5E
:102F900060E070E0CB01B8CF60EC72E0CE0101964A
:102FA0000E947B0EBE016F5F7F4F8CEB94E00E940E
:102FB0003A0D182FCE0101960E94A00D112341F168
:102FC00026E030E044E050E060EB74E0CE01019692
:102FD0000E940C0FBE016F5F7F4F8AEA94E00E944F
:102FE000550DCE0101960E94A00D8AEA94E00E9440
:102FF000D20C7093260460932504709310016093A3
:103000000F0180911101909112010E947A1475CDE7
:103010006CEB72E0CE0101960E947B0EBE016F5FE9
:103020007F4F8CEB94E00E943A0D182FCE01019651
:103030000E94A00D1123A9F143E050E060EB74E081
:10304000CE0101960E94580FBE016F5F7F4F8AEA42
:1030500094E00E94550DCE0101960E94A00D6AEAEF
:1030600074E0CE0101960E94F20ECE0101960E94FC
:10307000FE0DBC018EE994E00E94DB0ECE010196AC
:103080000E94A00D4091A2045091A3044115510546
:1030900009F4B7CF67E274E08EE994E00E94980CDF
:1030A000B0CF69EB72E0CE0101960E947B0EBE01AB
:1030B0006F5F7F4F8CEB94E00E943A0D182FCE018A
:1030C00001960E94A00D112309F48DC08091B404D3
:1030D0009091B504409708F00CC242E050E060EBDC
:1030E00074E0CE0101960E94580FBE016F5F7F4FC2
:1030F0008AEA94E00E94550DCE0101960E94A00D2F
:103100008091AA049091AB040097A9F10E945C2DD4
:1031100020E030E048EC52E40E9420320E94E23489
:103120006093310470933204809333049093340499
:103130008B019C0100591F452140310901341C4974
:1031400021053105E0F065E971E0CE0101960E94AC
:10315000FB0E6AEA74E0CE0101960E94320E6BE922
:1031600071E00E941C0EBC0182EC94E00E94DB0E18
:10317000CE0101966DCC60E070E0CB01C9CF0E941A
:10318000C13120E030E048EC52E40E947034AB01E1
:10319000BC0122E0CE0101960E94C70FBE016F5F05
:1031A0007F4F82EC94E00E94550DCE0101960E9463
:1031B000A00D6BEA71E0CE0101960E94FB0E62EC5D
:1031C00074E0CE0101960E94320E68EB71E00E941D
:1031D0001C0EBC0182EC94E00E94DB0ECE01019635
:1031E0000E94A00D0ECF6DEB71E0CE0101960E9402
:1031F000FB0EBE016F5F7F4F8CEB94E00E943A0D97
:10320000182FCE0101960E94A00D112339F06AEA11
:1032100072E082EC94E00E94560EABCE66EA72E059
:10322000CE0101960E947B0EBE016F5F7F4F8CEB3B
:1032300094E00E943A0D182FCE0101960E94A00D35
:10324000112309F45ACC43E050E06CEB74E0CE015A
:1032500007960E94580FBE01695F7F4FCE0101960D
:103260000E94F20ECE0101960E94FE0DBC018AEA78
:1032700094E00E94DB0ECE0101960E94A00DCE01CB
:1032800007960E94A00D6AEA74E0CE0149960E945A
:10329000F20E61EC71E0CE0101960E94FB0E8D8D65
:1032A0009E8D892BC9F1098D1A8D69817A81C8019A
:1032B0000E944D39009781F1FC01E01BF10B8F0159
:1032C000CE0101960E94A00D68E571E0CE01439603
:1032D0000E94FB0E68E571E0CE010D960E94FB0E88
:1032E00010161106E4F463EC71E0CE0101960E9421
:1032F000FB0ECE0101960E94640FCE0101960E9442
:10330000A00DCE010D960E94A00DCE0143960E9405
:10331000A00DCE01499639CE0FEF1FEFD1CFBE01E0
:10332000675E7F4FCE010D960E94DB0E10E000E03D
:103330002AEFA22EBB24BA9436E0932E89899A896B
:10334000009709F4C7C005301105D1F366E572E0B6
:10335000CE0101960E94FB0EBE016F5F7F4FCE0132
:103360000D960E943A0DF82ECE0101960E94A00DF6
:10337000F110A0C0EE24E394F12C970150E040E05E
:10338000BE01635F7F4FCE0107960E940C0FBE0106
:10339000695F7F4FCE0101960E94F20ECE01019629
:1033A0000E94FE0DBC01CE0143960E94DB0ECE01B1
:1033B00001960E94A00DCE0107960E94A00DBE01AD
:1033C0006D5E7F4FCE0107960E94F20E8B859C8525
:1033D000029708F473C066E572E0CE0101960E9480
:1033E000FB0EBE016F5F7F4FCE0107960E943A0D24
:1033F000D82ECE0101960E94A00DDD2009F45EC0FA
:1034000022E030E041E050E0BE01695F7F4FCE0135
:1034100001960E940C0FCE0101960E94D20C2B0146
:103420006B01CE0101960E94A00D57FE03C0FCE186
:10343000CF0ED11CB5016C197D09909E6001919E43
:10344000D00C1124F601EF58FB4F76876587CE012B
:1034500007960E94A00DB60166587B4F44E050E0ED
:10346000CE0143960E94980C0F5F1F4F89899A895D
:10347000E816F90640F5A701BE01635F7F4FCE0154
:1034800001960E94580FBE016F5F7F4FCE01439699
:103490000E94550DCE0101960E94A00DBE016D5EE9
:1034A0007F4FCE010D960E94DB0ECE010D960E943D
:1034B000DD0C44CF82E0E82EF12C5FCFCE010796E1
:1034C0000E94D20CBACF68E571E0CE010D960E9441
:1034D000A50E34CF00937304002341F081E0809364
:1034E00071048EE190E00E94A3140BCF109271043E
:1034F000F8CF80E007CB8F929F92AF92BF92CF928E
:10350000DF92EF92FF920F931F93CF93DF9300D040
:1035100000D000D0CDB7DEB720918602222309F477
:10352000A4C02091AB023091AC02243131050CF0E3
:103530009CC00091040110910501013C43E0140777
:103540000CF093C06C012F5F3F4F3093AC0220937F
:10355000AB020E945D0580907E0290907F02A09059
:103560008002B0908102681979098A099B090E943A
:10357000BF3120E030E04AE754E40E9470346093A9
:103580008202709383028093840290938502083CA8
:10359000110534F488EC90E09093050180930401C8
:1035A000809104019091050102E812E0FC01E258CB
:1035B000F2407F01C701800F911F9A838983F80130
:1035C00061918F01CE0101960E946114F2E00638EC
:1035D0001F0781F7E0900401F0900501C7010496F0
:1035E0009093050180930401B601CE0101960E94DB
:1035F000F20ECE0101960E94FE0DBC0182EC94E019
:103600000E94DB0ECE0101960E94A00D4091C604DF
:103610005091C7044115510531F067E872E082EC22
:1036200094E00E94980C8BEAC82E82E0D82E07E81E
:1036300012E09701235832407901C701800F911F92
:103640009A838983F80161918F01CE0101960E94CE
:103650006114C016D10689F780910401909105018B
:103660008496909305018093040126960FB6F894F2
:10367000DEBF0FBECDBFDF91CF911F910F91FF90A5
:10368000EF90DF90CF90BF90AF909F908F90089574
:103690002F923F924F925F926F927F928F929F9262
:1036A000AF92BF92CF92DF92EF92FF920F931F9350
:1036B000CF93DF93CDB7DEB7CC55D1090FB6F894D1
:1036C000DEBF0FBECDBF29966CAF7DAF8EAF9FAF73
:1036D000299725962CAF3DAF4EAF5FAF2597683E3B
:1036E00073408105910554F088E290E0A0E0B0E0DD
:1036F00029968CAF9DAFAEAFBFAF299725962CAD65
:103700003DAD4EAD5FAD25972115314E454F55402E
:1037100054F020E031EE45EF55E025962CAF3DAF5B
:103720004EAF5FAF259780910503882351F081E06C
:1037300090E0A0E0B0E025968CAF9DAFAEAFBFAFFC
:1037400025970E945D0569966CAF7DAF8EAF9FAFE8
:1037500069970E945D052D966CAF7DAF8EAF9FAFD0
:103760002D9769966CAD7DAD8EAD9FAD699728EEB6
:1037700033E040E050E00E94F7326D962CAF3DAF51
:103780004EAF5FAF6D97772473941E0197E0290EBB
:10379000311C2D966CAD7DAD8EAD9FAD2D9769968C
:1037A0002CAD3DAD4EAD5FAD6997621B730B840BC5
:1037B000950B25962CAD3DAD4EAD5FAD25976217AF
:1037C0007307840795070CF02CC30E94C13120E0D9
:1037D00030E04AE754E40E947034AB01BC0123E0BE
:1037E000CE0101960E94C70FBE016F5F7F4F8AEA2C
:1037F00094E00E94550DCE0101960E94A00D2596E1
:103800008CAD9DADAEADBFAD25970A97A105B105B5
:1038100024F518AA1FA61AAA19AA1CAA1BAA2AE0EC
:10382000AE014F5F5F4F6D966CAD7DAD8EAD9FADC0
:103830006D970E94A22DBE016F5F7F4FCE018F96C4
:103840000E94A50EBE01615D7F4F8AEA94E00E944E
:10385000550DCE018F960E94A00D809105038823FF
:1038600061F168E571E08AEA94E00E94A50E83E5C3
:103870000E94320262E389E194E00E9464090E949E
:10388000710783E50E94320266E070E083E590E014
:103890000E94B60908EF14E0C801885F94400F5FEA
:1038A0001F4F30912A0320912B03321701F10E9400
:1038B0001F02D8011D968C93EFCF65E871E0CE0111
:1038C00001960E94FB0E6AEA74E0CE0101960E9406
:1038D000320E6CE771E00E941C0EBC018AEA94E093
:1038E0000E94DB0ECE0101960E94A00DC0CF06976C
:1038F00029F01092F804B1E0B093F9040E94710726
:1039000080910605909107059A8389838091080527
:10391000909109059C838B8380910A0590910B05FA
:103920009E838D838E010F5F1F4F9AEF892E94E047
:10393000992E2E01E3E24E0E511C5201D8016D91D9
:103940007D918D01F401C190D190E190F1904F01F2
:10395000072E000C880B990B0E94C131A70196011C
:103960000E942032D5016D937D938D939D935D01CF
:103970000215130519F768E571E082EC94E00E94E6
:10398000A50E8201045F1F4FC12CD12C7601F201DC
:1039900081909190A190B1902F01A5019401C50152
:1039A000B4010E9420329B01AC01C701B6010E9404
:1039B00092336B017C0123E0B501A401CE01019695
:1039C0000E94C70FBE016F5F7F4FCE018F960E948E
:1039D000F20E60E771E0CE018F960E941C0EBC01D2
:1039E00082EC94E00E944F0ECE018F960E94A00DB3
:1039F000CE0101960E94A00D4016510641F6C70166
:103A0000B6010E94A2356B017C012DEC3CEC4CE42C
:103A10005FE30E943F3518160CF07AC12AE939E9B4
:103A200049E95FE3C701B6010E94BA3187FF70C15F
:103A3000772009F46DC18BA49CA4ADA4BEA44BA0B7
:103A40005CA06DA07EA0CFA0D8A4E9A4FAA420E039
:103A500030E0A901C501B4010E94BA31882309F4FC
:103A600044C1A3019201C301B2010E9420326196B8
:103A70006CAF7DAF8EAF9FAF6197A7019601C70175
:103A8000B6010E9420329B01AC0161966CAD7DAD08
:103A90008EAD9FAD61970E9492330E94A235A50121
:103AA00094010E94113420EE3EE245E652E40E9469
:103AB000203261966CAF7DAF8EAF9FAF619720E0F3
:103AC00030E0A901C701B6010E94BA31882309F488
:103AD00011C1A3019201C301B2010E942032659677
:103AE0006CAF7DAF8EAF9FAF6597A5019401C50107
:103AF000B4010E9420329B01AC0165966CAD7DAD96
:103B00008EAD9FAD65970E9492330E94A235A701AA
:103B100096010E94113420EE3EE245E652E40E94F6
:103B2000203265966CAF7DAF8EAF9FAF659720E07A
:103B300030E0A901C301B2010E94BA31882309F41F
:103B4000DEC0A5019401C501B4010E9420324B01E1
:103B50005C01A7019601C701B6010E9420329B01BA
:103B6000AC01C501B4010E9492330E94A235A301A9
:103B700092010E9411346B017C016AEA74E0CE016B
:103B800001960E94F20E6AED71E0CE0101960E944C
:103B90001C0EBC0182EC94E00E94DB0ECE0101966B
:103BA0000E94A00D62EC74E0CE0101960E94F20E1C
:103BB000CE0101960E94A809CE0101960E94A00D97
:103BC00021E061964CAD5DAD6EAD7FAD6197CE01EC
:103BD000CB960E94C70F21E065964CAD5DAD6EADF2
:103BE0007FAD6597CE01C5960E94C70F20EE3EE2DD
:103BF00045E652E4C701B6010E942032AB01BC0188
:103C000021E0CE0101960E94C70FBE016F5F7F4F7A
:103C1000CE018F960E94F20E60E771E0CE018F9682
:103C20000E941C0EBE016B5C7F4F0E94320E60E74B
:103C300071E00E941C0EBE01655C7F4F0E94320E37
:103C4000BC0182EC94E00E94DB0ECE018F960E94B4
:103C5000A00DCE0101960E94A00DCE01C5960E9436
:103C6000A00DCE01CB960E94A00D62EC74E0CE01B7
:103C700001960E94F20ECE0101960E94640FCE01C1
:103C800001960E94A00D772473940E945D05DC01CB
:103C9000CB012D962CAD3DAD4EAD5FAD2D97821B6A
:103CA000930BA40BB50B29962CAD3DAD4EAD5FAD7E
:103CB000299782179307A407B50744F4281B390BEB
:103CC0004A0B5B0BCA01B9010E9438040E945D05D2
:103CD0002D966CAF7DAF8EAF9FAF2D9768E571E0ED
:103CE00082EC94E00E94A50E54CD6BED7FE089EC50
:103CF0009FE3D9CE6BED7FE089EC9FE30CCF8BED9A
:103D0000C82E8FE0D82E89ECE82E8FE3F82E35CF21
:103D100062EF71E0CE0101960E94FB0E62EC74E04E
:103D2000CE0101960E94320EBC0182EC94E00E940A
:103D3000DB0ECE0101960E94A00D62EC74E0CE0174
:103D400001960E94F20ECE0101960E94640FCE01F0
:103D500001960E94A00D62EC74E0CE0101960E94D3
:103D6000F20ECE0101960E947B1ACE0101960E94AE
:103D7000A00D23E0B701A601CE018F960E94C70FC8
:103D80006FEF71E0CE0101960E94FB0EBE01615DF6
:103D90007F4FCE0101960E94320E62E072E00E94D7
:103DA0001C0EBC0182EC94E00E94DB0ECE01019659
:103DB0000E94A00DCE018F960E94A00D62EC74E0CF
:103DC000CE0101960E94F20ECE0101960E947B1A4E
:103DD000CE0101960E94A00D6AEA74E0CE01019620
:103DE0000E94F20E62EC74E0CE0101960E94320E47
:103DF000BC0182EC94E00E94DB0ECE0101960E9491
:103E0000A00D62EC74E0CE0101960E94F20ECE018C
:103E100001960E94640FCE0101960E94A00D712CA4
:103E200034CFC45ADF4F0FB6F894DEBF0FBECDBFFC
:103E3000DF91CF911F910F91FF90EF90DF90CF9086
:103E4000BF90AF909F908F907F906F905F904F90BA
:103E50003F902F9008954F925F926F927F928F9232
:103E60009F92AF92BF92CF92DF92EF92FF920F9309
:103E70001F93CF93DF93CDB7DEB7E9970FB6F894D2
:103E8000DEBF0FBECDBF7C0168E571E082EC94E03F
:103E90000E94A50EC7010596059768F0809105035D
:103EA000811109C02CEEE2162FEFF20624F0F092F9
:103EB0000003E092FF02F7017A96E432F10508F080
:103EC00035C7EB59F04E0C943037232696261F2623
:103ED0009626962696269626962696269626962602
:103EE000282228222822891F2822282228228322C9
:103EF00028222822862295229822962628222822C5
:103F0000A6221D24282240255E2568252822282255
:103F1000E62560E08FE00E94E203E7EAF3E0E49147
:103F2000ED8BE3E9F3E0E491F0E0EE0FFF1FE658DC
:103F3000FC4F859194919F8B8E8B18A21AA219A287
:103F4000CE01459698878F831D821E82198289E053
:103F50008A8381E08B838C831C8A1B8A1F8E1E8E32
:103F60001D8E1C8E1B8E1A8E198E188E01E0BE01BE
:103F70006D5D7F4F8F8198850E94DC0B882309F44B
:103F80005BC067E0CE0183960E9469059AA58913FC
:103F9000EECF898181111DC08F8198850E942606F0
:103FA000BE016D5D7F4F8F8198850E94070640E0BE
:103FB00064EB8F8198850E94D3058F8198850E943C
:103FC0008005182F8F8198850E942606111101C047
:103FD00009831A818BA1803109F4AFC6BE016D5DE2
:103FE0007F4FCE0101960E94BE06811790F48A8110
:103FF0008A838D818F5F8D838BA1883231F0B0F4FD
:10400000803119F0823209F0B2CF8E818F5F8E83BA
:10401000AECF8BA1803111F48CE0EACFBE016D5D93
:104020007F4FCE0101960E94BE06E2CF8B3369F32B
:10403000823409F09CCFE9CF8F8198850E942606B3
:1040400040E06CEC8F8198850E94D305498164E43F
:104050008F8198850E94D3058B81882379F1EA812D
:10406000E9509EEEC92E92E0D92EE33038F4F0E00C
:10407000EE0FFF1FE25EFE4FC080D1808C8188234F
:1040800009F461C0898181115EC00E945D054B0108
:104090005C010D2C000CEE08FF088F8198850E94B2
:1040A0008005813059F00E945D056C197D098E09EB
:1040B0009F09681579058A059B0578F38CE08A834A
:1040C000F12CE12C0FE5BFE7DB2E1FE1C12E8FE3C2
:1040D000B82E8D818E151F0409F00CF499C04E2D59
:1040E000BE01645D7F4FCE0101960E945C0C1A8177
:1040F0001D3080F11CE08CA5803181F1BE01645D32
:104100007F4FCE0101960E94BE06811709F478C048
:10411000AE014D5D5F4FBE01645D7F4FCE010196E4
:104120000E945E06882309F46BC08CA5803109F4D7
:1041300067C01B3009F468C01C3091F01A3009F0D8
:1041400065C0BFA20EC0B601DD0C880B990B0E94A2
:104150003804B4CF193078F619E0CDCF8CE0D5CF44
:10416000DFA28F8198850E942606BE01645D7F4F85
:104170008F8198850E94070640E06EE48F819885C4
:104180000E94D30540E06DA18F8198850E94D305E0
:1041900040E06EA18F8198850E94D3058CA5803167
:1041A00031F040E06FA18F8198850E94D3058F8107
:1041B00098850E942606BE01645D7F4F8F81988599
:1041C0000E940706498168E48F8198850E94D30583
:1041D00064E170E080E090E00E94380489818823E7
:1041E00031F06AE070E080E090E00E9438048F8156
:1041F00098850E9426068A81811708F4812F8A8378
:104200003FEFE31AF30A65CF0FA3ABCFCFA2A9CF3D
:104210000E8110E06DE472E00115110509F488C506
:1042200068E571E082EC94E00E94A50E680105301B
:1042300011051CF0A4E0CA2ED12CF1E5AF2EF4E05C
:10424000BF2EF12CE12C4E2DBE01645D7F4FCE01BF
:1042500001960E945C0C81113DC020E030E04EEFE1
:1042600052ECF50161917191819191915F010E94F0
:1042700092332B013C01FFEFEF1AFF0A20E030E000
:104280004CEF52EC0E94BA3187FF70C0B701CE01EB
:104290008C960E94AF0E65E072E0CE0183960E947C
:1042A000FB0EBE01645D7F4FCE0183960E94320EED
:1042B00067E072E00E941C0EBC0182EC94E00E9458
:1042C0004F0ECE0183960E94A00DCE018C960E94C7
:1042D000A00D98C0AE014D5D5F4FBE01645D7F4F84
:1042E000CE0101960E945E06882309F4B6CF6CA128
:1042F00070E0762F6627770F770F770F2BA148E0B6
:10430000249F90011124262B372B8CA58031D1F4CA
:104310006AA570E089A5FB01E81BF109CF0196951C
:10432000982F8827979587950E941C37CB01409737
:10433000B90153E0660F771F5A95E1F760789C0149
:10434000260F371F2138F4EE3F070CF486CFB90152
:10435000330F880B990B0E94C13120E030E040E020
:104360005CE30E9420329B01AC017BCF22E0B301D1
:10437000A201CE010330110509F4A9C0C4960E9420
:10438000C70FB701CE018C960E94AF0E65E072E0B8
:10439000CE0183960E94FB0EBE01645D7F4FCE016D
:1043A00083960E94320E6BE172E00E941C0EBE01E9
:1043B0006C5C7F4F0E94320EBC0184EA94E00E9444
:1043C000DB0ECE0183960E94A00DCE018C960E943A
:1043D000A00DCE01C4960E94A00D64EA74E0CE0147
:1043E00083960E94F20E60E771E0CE0183960E94F0
:1043F0001C0EBC0182EC94E00E944F0ECE0183960D
:104400000E94A00DEC14FD040CF41DCF82EC94E08E
:104410000E94DD0C03301105A9F463E172E0CE01C6
:1044200083960E94FB0E62EC74E0CE0183960E949C
:10443000320EBC0182EC94E00E94DB0ECE0183962A
:104440000E94A00D6DE172E082EC94E00E94450EA6
:104450008091C6049091C704892BE1F062EC74E06E
:10446000CE0101960E94F20ECE0101960E94640FC9
:10447000CE0101960E94A00D62EC74E0CE0101967F
:104480000E94F20ECE0101960E947B1ACE01019687
:104490000E94A00D64E670E080E090E00E94380485
:1044A000E9960FB6F894DEBF0FBECDBFDF91CF9176
:1044B0001F910F91FF90EF90DF90CF90BF90AF9042
:1044C0009F908F907F906F905F904F90089583960C
:1044D0000E94C70FBE016D5D7F4FCE018C960E947A
:1044E000F20E60E771E0CE018C960E941C0EBC01BA
:1044F00082EC94E00E944F0ECE018C960E94A00D9B
:10450000CE018396E4CE0E945D05A2CF8091050383
:10451000882321F082EC94E00E94750268EC70E040
:1045200080E090E00E94380493CF1092050390CF72
:1045300081E080930503809379048091FF0290913C
:1045400000039093FE028093FD0282CF64E670E048
:1045500080E090E00E94380480910F01909110015A
:104560000B9731F580911905882309F0F89482E1C1
:104570000E946B048C0180911905882309F07894BE
:104580000115110509F4ADC080E090ECA9E7B4EC89
:1045900080930C0590930D05A0930E05B0930F0525
:1045A0008093100590931105A0931205B093130505
:1045B00080910F0190911001469731F58091190576
:1045C000882309F0F89481E00E946B048C018091AB
:1045D0001905882309F078940115110509F4E2C042
:1045E00080E090ECA9E7B4EC80930C0590930D0566
:1045F000A0930E05B0930F058093100590931105BD
:10460000A0931205B093130564E670E080E090E09B
:104610000E943804012B09F01BCF409110055091E6
:104620001105609112057091130521E0CE014596A8
:104630000E94C70F60E372E0CE0101960E94FB0E5C
:10464000BE016B5E7F4FCE0101960E94320E63E386
:1046500072E00E941C0EBC0182EC94E00E94DB0E12
:10466000CE0101960E94A00D40910C0550910D05C0
:1046700060910E0570910F0521E0CE0101960E9418
:10468000C70FBE016F5F7F4FCE0145960E94550D4B
:10469000CE0101960E94A00D67E372E0CE01019663
:1046A0000E94FB0EBE016B5E7F4FCE0101960E9401
:1046B000320E6AE372E00E941C0EBC0182EC94E0B0
:1046C0000E944F0ECE0101960E94A00D64E670E09C
:1046D00080E090E00E943804CE0145960E94A00D33
:1046E000B7CE10911405E09015056E2D70E090E0A6
:1046F00080E00E94C1312DEC3CEC4CEC5DE30E946B
:1047000020324B015C01612F70E090E080E00E945C
:10471000C1319B01AC01C501B4010E949233609389
:104720000C0570930D0580930E0590930F05009175
:104730001605F0901705602F6F7770E090E080E02D
:104740000E94C1314B015C016F2D70E090E080E070
:104750000E94C1312DEC3CEC4CEC5DE30E94203218
:104760009B01AC01C501B4010E94923307FD18C042
:1047700060931005709311058093120590931305B3
:10478000812F8E0D800F8F0D01E010E090911805A4
:10479000891302C010E000E011950195110908CFBE
:1047A0009058E6CF109115050091140560911405FD
:1047B0007091150576276727762790E080E00E94A4
:1047C000BF312DEC3CEC4CEC5DE30E942032609359
:1047D0000C0570930D0580930E0590930F05E090E6
:1047E0001705F09016056F2D6F77762F6E2D90E0E0
:1047F00080E00E94BF312DEC3CEC4CEC5DE30E946C
:104800002032F7FC18C06093100570931105809357
:10481000120590931305812F800F8E0D8F0D01E0EF
:1048200010E090911805891302C010E000E0119586
:1048300001951109E9CE9058E6CF80910E018823A9
:1048400009F406CE0E94170A6B017C010E94FF0941
:104850009C0150E040E08091F6049091F704281B01
:10486000390B41095109A091F404B091F5040E945B
:1048700016334B015C019FE0B594A79497948794FD
:104880009A95D1F76091EE047091EF04072E000C19
:10489000880B990B2BE0660F771F881F991F2A95AD
:1048A000D1F72091F0043091F104032E000C440B59
:1048B000550B280D391D4A1D5B1D0E94F732CA0198
:1048C000B901680D791D8A1D9B1D685F7F4F8F4F51
:1048D0009F4F34E095958795779567953A95D1F7F1
:1048E0000E94C1312B013C0160913104709132046E
:1048F00080913304909134040E94C1314B015C01DA
:104900000E94170A0E94C131A50194010E947034CF
:1049100021E03EED42E45EE30E944C354B015C0138
:10492000C701B6010E94C13120E030E048EC52E4FA
:104930000E947034AB01BC0122E0CE0101960E94BE
:10494000C70FBE016F5F7F4F84EA94E00E94550D50
:10495000CE0101960E94A00D69EB71E084EA94E01B
:104960000E94450E64EA74E08AEA94E00E94DB0E3D
:1049700068E971E0CE0101960E94FB0E64EA74E0E2
:10498000CE0101960E94320EBC0184EA94E00E949E
:10499000DB0ECE0101960E94A00D60E672E082EC73
:1049A00094E00E94560E20E030E040E251E4C30162
:1049B000B2010E947034AB01BC0121E0CE0101962E
:1049C0000E94C70FBE016F5F7F4F82EC94E00E9490
:1049D0004F0ECE0101960E94A00D6CE372E082ECB6
:1049E00094E00E94450EA501940160E070E080E82B
:1049F0009FE30E94913320E03AE24DE257E40E94A7
:104A00002032AB01BC0121E0CE0145960E94C70FC8
:104A1000BE016B5E7F4FCE0101960E94F20E62E4F2
:104A200072E0CE0101960E941C0EBC0182EC94E063
:104A30000E944F0ECE0101960E94A00DCE01459618
:104A40000E94A00D64EA74E0CE0101960E94F20E6D
:104A500060E771E0CE0101960E941C0E62EC74E0EA
:104A60000E94320EBC0182EC94E00E94DB0ECE016B
:104A700001960E94A00D65E070E080E090E052CDCC
:104A800081E0809317010E94EE048C0163E672E0DE
:104A900082EC94E00E94560E60E074E0601B710BA3
:104AA000CE0101960E94AF0EBE016F5F7F4F82EC78
:104AB00094E00E944F0ECE01019610CE63E772E0A3
:104AC00082EC94E00E94560E0E94EE04BC01E8CFF6
:104AD00080910E01882309F4BBCC809105038823C3
:104AE00029F082E090E00E945511B2CC20E030E045
:104AF0004AE754E460910001709101018091020144
:104B0000909103010E9420320E94E2344B015C012B
:104B100020E030E04AE754E4609113017091140101
:104B200080911501909116010E9420320E94E2347A
:104B30006B017C0129EEC21623E0D206E104F104E8
:104B40002CF084E1C82ED12CE12CF12C0E945D05C3
:104B500060937A0270937B0280937C0290937D0233
:104B60000E945D052B013C0180917A0290917B02AD
:104B7000A0917C02B0917D02A3019201281B390B08
:104B80004A0B5B0BDA01C90188159905AA05BB051B
:104B90000CF05ECC83E090E00E9455110E945D0510
:104BA000DC01CB0184199509A609B7098C159D056F
:104BB000AE05BF05ACF6A7019601281B390B4A0BC1
:104BC0005B0BCA01B9010E943804CACF80910E0163
:104BD000882309F43DCC80910503882359F021E016
:104BE00030E040E050E06AE070E080E090E00E9459
:104BF000481B2ECC20E030E04AE754E460910001ED
:104C00007091010180910201909103010E94203274
:104C10000E94E2346B017C0120E030E04AE754E47A
:104C2000609113017091140180911501909116010A
:104C30000E9420320E94E234A7019601D8CFF0E012
:104C4000E0E0099505CC8091730418160CF055C06E
:104C500081E0809371046CE872E082EC94E00E9441
:104C6000560E80917104882309F44AC064E472E00E
:104C7000CE0101960E94FB0E62EC74E0CE0101961B
:104C80000E94320EBC0182EC94E00E94DB0ECE0149
:104C900001960E94A00D62EC74E0CE0101960E9484
:104CA000F20ECE0101960E94640FCE0101960E9481
:104CB000A00D68EE73E080E090E00E9438048091DF
:104CC000710481110E94A12668E571E082EC94E0F4
:104CD0000E94A50E80910503809379048111B8CBC1
:104CE00065E572E086EB94E00E94A50E86EE9FEFEC
:104CF000909300038093FF02ABCB10927104ABCF73
:104D00006CE472E0CE0101960E94FB0E62EC74E04E
:104D1000CE0101960E94320EBC0182EC94E00E940A
:104D2000DB0ECE0101960E94A00DD4CF6EE772E09B
:104D300082EC94E00E94560E8BCB1D3008F057C9D0
:104D40006BC90F931F93CF93DF9301E714E0D0E07B
:104D5000C0E00A5F1F4F80917304082E000C990B6E
:104D6000C817D9076CF4F801878190850E942B1F22
:104D700068EE73E080E090E00E9438042196E9CF6D
:104D8000DF91CF911F910F9108951F920F920FB64F
:104D90000F9211242F933F934F935F936F937F93C1
:104DA0008F939F93AF93BF93EF93FF938CE793E021
:104DB0000E94D802FF91EF91BF91AF919F918F9187
:104DC0007F916F915F914F913F912F910F900FBE07
:104DD0000F901F9018951F920F920FB60F921124EB
:104DE0002F938F939F93EF93FF93E0918C03F09118
:104DF0008D038081E0919203F091930382FD1BC0AB
:104E00009081809195038F5F8F7320919603821715
:104E100041F0E0919503F0E0E458FC4F958F8093CA
:104E20009503FF91EF919F918F912F910F900FBE5E
:104E30000F901F9018958081F4CF1F920F920FB69C
:104E40000F9211242F933F938F939F93AF93BF9310
:104E50008091F2029091F302A091F402B091F502D8
:104E60003091F10223E0230F2D3758F50196A11D53
:104E7000B11D2093F1028093F2029093F302A0936C
:104E8000F402B093F5028091F6029091F702A0919E
:104E9000F802B091F9020196A11DB11D8093F602AE
:104EA0009093F702A093F802B093F902BF91AF91EB
:104EB0009F918F913F912F910F900FBE0F901F9058
:104EC000189526E8230F0296A11DB11DD2CF1F927F
:104ED0000F920FB60F9211242F933F934F935F932E
:104EE0006F937F938F939F93AF93BF93EF93FF93B2
:104EF0008091B900887F803609F44AC0F0F5883285
:104F000009F4A7C018F5803109F49BC0B8F48823D0
:104F100009F4F9C0883009F494C0FF91EF91BF9172
:104F2000AF919F918F917F916F915F914F913F9141
:104F30002F910F900FBE0F901F901895883109F494
:104F400088C0803251F78093500314C0803409F434
:104F50009DC040F48033B9F38833F9F68093500351
:104F600085ECB0C0803509F485C0883509F496C059
:104F7000883499F60E941D11D0CF883909F48CC06D
:104F800038F5883729F050F4883611F0803729F643
:104F900083E0809352031092F00257C0883809F4DE
:104FA0007BC0803919F0803809F0B7CF8091F002CA
:104FB000803208F071C0E091F00281E08E0F8093A2
:104FC000F0028091BB00F0E0E053FD4F80833DC0D4
:104FD000803B39F0E0F4803A09F479C0883A09F06E
:104FE0009CCF84E0809352031092CF021092CE02A5
:104FF000E0910803F091090309958091CE02811197
:105000000FC081E08093CE021092AE0209C0803CB6
:1050100009F4A6CF883C09F4A3CF883B09F07DCFE3
:10502000E091CF0281E08E0F8093CF02F0E0E25555
:10503000FD4F80818093BB009091CF028091CE0282
:1050400029C080912D038093BB0085EC8093BC0028
:1050500064CF90914F0380914E03981758F5E091DB
:105060004F0381E08E0F80934F03F0E0E25DFC4F31
:105070008081E9CFE0914F0381E08E0F80934F0351
:105080008091BB00F0E0E25DFC4F808390914F0384
:1050900080914E039817C8F285E8D8CFE0914F036E
:1050A00081E08E0F80934F038091BB00F0E0E25DC2
:1050B000FC4F80838091510381115CCF81E080930C
:1050C0002C0384EA8093BC001092520326CF85EC17
:1050D0008093BC00109252038091F002803230F431
:1050E000E091F002F0E0E053FD4F10826091F00299
:1050F00070E0E0910603F091070380ED92E00995DE
:105100001092F0020ACF1092500334CFCF93DF9366
:10511000ECE7F3E01382128288EE93E0A0E0B0E0C7
:1051200084839583A683B78328E231E0318320838B
:1051300025EC30E03587248724EC30E0378726875C
:1051400020EC30E0318B208B21EC30E0338B228B54
:1051500022EC30E0358B248B26EC30E0378B268B2D
:10516000118E128E138E148EE9E1F4E013821282F6
:1051700084839583A683B7838AE391E091838083B8
:1051800010921905E8EFF4E0C1E0C083118283ECCE
:105190009BEAA6E7BBE382839383A483B58388ED70
:1051A0009BE6A6E7BBE386839783A087B18782EF60
:1051B00094EEA4E6BBE382879387A487B587E8ECE7
:1051C000F4E08CE491E0918380838FEF9FEFDC012A
:1051D000858B968BA78BB08F68E571E082EC94E0AD
:1051E0000E94FB0E68E571E08CEB94E00E94FB0EE0
:1051F00068E571E086EB94E00E94FB0E68E571E0E3
:1052000080EB94E00E94FB0E68E571E08AEA94E08E
:105210000E94FB0E68E571E084EA94E00E94FB0EB8
:1052200068E572E08EE994E00E94FB0E6FE572E0A3
:1052300088E994E00E94FB0EE1E7F4E0108285E04B
:10524000818312821482138216821582178210863D
:10525000E5E2F4E086E190E0918380838CE79CE8CE
:10526000A1E0B0E084879587A687B78781EA97E6B3
:10527000A3E3BDEB808B918BA28BB38B86E696E686
:10528000A6EABFE3848B958BA68BB78BC0A389E17D
:1052900090E092A381A3C3A380E090E4ACE1B5E4E5
:1052A00084A395A3A6A3B7A310A611A612A613A61E
:1052B000A1E5B4E080E1ED0119928A95E9F714AE19
:1052C00015AE16AE17AE10926504109266041092D9
:1052D0006704109268041092690410926A04109294
:1052E0006B0410926C0410926D0410926E04109274
:1052F0006F0410927004DF91CF910895CF93DF93E4
:10530000CDB7DEB7AE970FB6F894DEBF0FBECDBFF8
:10531000789484B5826084BD84B5816084BD85B590
:10532000826085BD85B5816085BD80916E0081609C
:1053300080936E0010928100809181008260809342
:105340008100809181008160809381008091800044
:105350008160809380008091B10084608093B1006F
:105360008091B00081608093B00080917A00846069
:1053700080937A0080917A00826080937A00809195
:105380007A00816080937A0080917A0080688093AF
:105390007A001092C10061E08EE00E94E203E09189
:1053A0008C03F0918D0382E08083E0918803F0917B
:1053B00089031082E0918A03F0918B038FEC808344
:1053C00010929403E0919003F091910386E0808322
:1053D000E0918E03F0918F03808180618083E09162
:1053E0008E03F0918F03808188608083E0918E032B
:1053F000F0918F03808180688083E0918E03F0912B
:105400008F0380818F7D808361E080E10E94E203D1
:1054100060E080E10E94B40361E08EE00E94B4038A
:1054200068EC70E080E090E00E94380484E690E050
:1054300090931201809311010E94E1328093FA024D
:1054400085E690E00E94E1328093FB020091FA022F
:105450001091FB02B801012E000C880B990B0E94E1
:10546000C1319B01AC010E94E635811106C00B5091
:1054700011090C30110508F4B8C084E690E00E94D0
:105480007A1431E7E32E34E0F32E67010EE110E0E9
:10549000C8010E94E132F60181936F010F5F1F4F37
:1054A00007321105A9F710917204612F012E000C2B
:1054B000770B880B990B0E94C1319B01AC010E94B4
:1054C000E635811103C0153009F4BAC08EE190E0D1
:1054D0000E94A31468EC70E080E090E00E94380421
:1054E00067E573E082EC94E00E94560E62EC74E093
:1054F000CE0101960E94F20ECE0101960E94640F29
:10550000CE0101960E94A00D0E94390764E670E06A
:1055100080E090E00E94380483E08093E1040E94E0
:10552000390780ED0E94BD09853509F497C06BE409
:1055300073E082EC94E00E94560E10920E0162EC31
:1055400074E0CE0101960E94F20ECE0101960E94F7
:10555000640FCE0101960E94A00DF12CE12C9AE27D
:10556000C92ED12C28EE422E23E0522E612C712C14
:1055700001E080E0A82E80E0B82E68E571E0CE0161
:1055800089960E94FB0E10E08CE793E00E94B8021F
:10559000181619060CF00CC111110AC18CE793E022
:1055A0000E9496028A3009F0B3C11091FC021123C7
:1055B00009F4C3C18091B4049091B504892B09F416
:1055C000B5C168E672E0CE0101960E94FB0EBE01F5
:1055D000675D7F4FCE0101960E94320E0E947502D8
:1055E000CE0101960E94A00DA1C145E2E42E44E047
:1055F000F42E04E610E0C8010E94E132F701819325
:105600007F010F5F1F4F003B1105A9F78091250413
:10561000909126049093100180930F0167E274E04B
:10562000CE0101960E94FB0EBE016F5F7F4F8EE997
:1056300094E00E94550DCE0101960E94A00D21CF4D
:105640000EE110E0C8010E94E132F70181937F0171
:105650000F5F1F4F05341105A9F73CCF8AEA0E945E
:10566000DA099093E3048093E2048CEA0E94DA0959
:105670009093E5048093E4048EEA0E94DA09909303
:10568000E7048093E60480EB0E94DA099093F30428
:105690008093F20482EB0E94DA099093F5048093E0
:1056A000F40484EB0E94DA099093F7048093F604E3
:1056B00086EB0E94DA099093E9048093E80488EB72
:1056C0000E94DA099093EB048093EA048AEB0E942B
:1056D000DA099093ED048093EC048CEB0E94DA09D4
:1056E0009093EF048093EE048EEB0E94DA0990937E
:1056F000F1048093F00464EF71E080E090E00E9498
:1057000038040E94390780E00E94930980E10E94DA
:10571000930988E00E9493090E9439078EE10E9454
:10572000320262E089E194E00E94640960E089E16C
:1057300094E00E9464090E9471078EE10E94320287
:1057400061E089E194E00E94640960E289E194E00B
:105750000E9464090E94710780E290E09093CC045B
:105760008093CB0480E090E8A9E8B4E480930A0138
:1057700090930B01A0930C01B0930D0180E090E099
:10578000A5E7B4E48093060190930701A093080174
:10579000B0930901BE016F5F7F4F88EC94E00E94D7
:1057A000FD0F64EF71E080E090E00E943804D5CEF8
:1057B0008DA59EA5892B51F08CE793E00E944703AD
:1057C00064E170E080E090E00E943804BE01675D13
:1057D0007F4F80EB94E00E94550DCE0189960E9488
:1057E000A00D68E571E082EC94E00E94A50E809126
:1057F000B4049091B5048130910509F0C6C060EB06
:1058000074E08CEB94E00E94DB0E0E94BB0C6CEB0E
:1058100074E0CE0101960E94F20E8D819E81892B4B
:1058200009F4A5C0E981FA81309709F4A0C080810C
:10583000823409F484C0833409F48EC0813409F0C1
:1058400096C061E772E080EB94E00E94A50ECE0165
:1058500001960E94A00D80EB94E00E94D20CCB0137
:105860000E942B1F80910503882309F43FC00E94EA
:105870005D05A30192010E946033CA01B9010E9433
:10588000BF312091010330910203409103035091F5
:1058900004030E949133209113013091140140912F
:1058A0001501509116010E943F351816FCF48091A5
:1058B000FF02909100034A9609F4B8C08091FD025E
:1058C0009091FE020E942B1F0E945D05A301920190
:1058D0000E946033CA01B9010E94BF316093010385
:1058E0007093020380930303909304036AE070E0D3
:1058F00080E090E00E943804A114B10409F43DCE88
:105900000E94C402882309F438CE0E94000031CEE0
:105910008D3009F44ACE89831A8241E050E0BE01FD
:105920006F5F7F4FCE0189960E94D20D6AE070E0D2
:1059300080E090E00E94380427CE11E0F7CF64E7C2
:1059400072E080EB94E00E94A50E109205038CEFAC
:105950009FEF0E942B1F7BCF67E772E080EB94E004
:105960000E94A50E009305038DEF9FEFF2CFBE01BD
:105970006F5F7F4F80EB94E00E94DB0E6AE070E087
:1059800080E090E00E94380462CF049768F566E5F5
:1059900072E0CE0101960E94FB0EBE016F5F7F4F49
:1059A00080EB94E00E943A0D182FCE0101960E94E0
:1059B000A00D1123C9F08091B4049091B504029711
:1059C00088F0E091B004F091B104309759F08181F2
:1059D00080330CF4845E9601281B310987FD3395D2
:1059E000C9013ECF80E0F6CF60EB74E08CEB94E031
:1059F0000E94DB0E0E94BB0C63E773E0CE010196B0
:105A00000E947B0EBE016F5F7F4F8CEB94E00E9483
:105A10003A0D182FCE0101960E94A00D112319F006
:105A2000F70109951FCF0E94CC141CCF80917104FF
:105A3000882309F449CF0E94A12646CF88E994E043
:105A40000E94A00D8EE994E00E94A00D84EA94E0EB
:105A50000E94A00D8AEA94E00E94A00D80EB94E0E1
:105A60000E94A00D86EB94E00E94A00D8CEB94E0C8
:105A70000E94A00D82EC94E00C94A00DEF920F9385
:105A80001F93CF93DF93E80134E047FD34E1042E08
:105A9000000C550B57FF03C0519541955109E32E5A
:105AA000022F242FAE010E94022ECE01DF91CF9152
:105AB0001F910F91EF900895662777270C94612F1F
:105AC0001F93FC0199278827BC01E894119110329B
:105AD000E9F3193010F01E30C8F31B3251F01D32BB
:105AE00049F4689406C00E94B12D610F711D811D9B
:105AF000911D119110531A30B0F33EF4909580959A
:105B0000709561957F4F8F4F9F4F1F910895FB01B7
:105B1000DC0105900D920020E1F70895FC0105904D
:105B20000020E9F7809590958E0F9F1F0895BB2761
:105B30004A3031F4992322F4BDE2909581959F4F2C
:105B40000C94E92DBB272A3051F4992342F4BDE28D
:105B500090958095709561957F4F8F4F9F4F0C94D6
:105B6000C72D592F482F372F262F660F771F881FD5
:105B7000991F660F771F881F991F620F731F841F5D
:105B8000951F660F771F881F991F0895BB27FA017D
:105B9000A62F6217710581059105330B30FB66F066
:105BA000AA27660F771F881F991FAA1FA21710F038
:105BB000A21B63953850A9F7A05DAA3308F0A95D30
:105BC000A19336F7B111B1931082CA010C94AA3196
:105BD000BB27FB015527AA27880F991FAA1FA417C7
:105BE00010F0A41B83955051B9F7A05DAA3308F0BB
:105BF000A95DA193009779F7B111B1931192CB01EF
:105C00000C94AA31A9E0B0E0E8E0FEE20C942F3356
:105C10006A01F22EB02E102FFBE3AF2EA01608F46F
:105C20001BE31F5F012F27E0AE014F5F5F4F0E9414
:105C3000B130BC018981982F9970913009F43FC02F
:105C40009BE2E1FC04C09E2D9170E0FC3AC05E2D09
:105C50005071E82FE87083FF46C084E0911101C0C5
:105C600083E0EF2DE81B8F1508F0E0E0D6018E2FC2
:105C700020E2552351F1992329F0D6019C93C601C6
:105C800001966C0196012D5F3F4FE2FE24C08EE429
:105C9000D6018C9391E411969C93119712968C9354
:105CA000D9018E2F90E281111BC0E20FF32FF11D5D
:105CB00010828EEF9FEF2996ECE00C944B339DE21F
:105CC000C6CF90E2C4CF2D9381508111FCCFCE0E70
:105CD000D11CE0E0D0CF8EE6D6018C9391E6DBCFED
:105CE0009D938150E0CF482F447082FF3DC084E0F7
:105CF000911101C083E08F1510F4EF2DE81BD60140
:105D00008E2F20E2552309F1992329F0D6019C9387
:105D1000C60101966C0196012D5F3F4FE2FE1BC04C
:105D200089E4D6018C938EE411968C93119786E4C6
:105D300012968C93D9018E2F90E2882309F4B5CF67
:105D40009D938150FACF2D9381508111FCCFCE0EBF
:105D5000D11CE0E0D9CF89E6D6018C938EE611966E
:105D60008C93119786E6E4CF9B0177FF02C030E069
:105D700020E0A1E0B0E0911102C0B0E0A0E0F901A4
:105D80003196AE0FBF1F8B2C912CBB2009F461C044
:105D90005401EFEFAE1ABE0AAA0DBB1DFA161B0680
:105DA00019F014F04F2D4A1B511188C0E3FC59C063
:105DB0007601A42FB0E2A1114FC0C40ED11C9923CB
:105DC00009F45BC040E0D6011196F60190836D01A5
:105DD000552309F448C0012F060F9A81582F50719E
:105DE00084FF03C0913309F4015010160CF047C032
:105DF000093008F008E0EEE2FE2E5B01A01AB108BF
:105E000085019194819491082F3F320729F4D6019E
:105E1000FC92F60131966F016217730794F1021735
:105E200013077CF5DB01A21BB30BAA24A394B12CAE
:105E3000AC0EBD1EAA0DBB1D11968C9121503109CF
:105E4000D601119628153905F4F0F60180836D010D
:105E5000DBCFB12CA12CA0CFF701B1937F01A150D2
:105E6000AACF9111B0CFD601942F50E302C05D9319
:105E700091509111FCCFC40ED11C40E0ACCF01E099
:105E8000BACF80E3DBCF6217730731F4963388F41F
:105E9000953311F4552369F0F6018083FD01842FB9
:105EA00090E2811108C0A40FB11D1C9290E080E027
:105EB00002CF81E3F1CF91938150F3CF911183CF42
:105EC0008ACFB0E0A0E0E7E6FFE20C942F335C015C
:105ED0007B016115710519F0DB018D939C938501A0
:105EE0000F5F1F4FF501D0818D2F90E00E94893107
:105EF0006C01892BB9F5DD32B9F50F5F1F4FD50164
:105F00001196DC91C1E05801F1E0AF1AB10843E00D
:105F100050E060E271E0C5010E949231892B69F581
:105F2000680182E0C80ED11C45E050E06BE171E0F1
:105F3000C6010E949231892B21F4680197E0C90EB5
:105F4000D11CE114F10419F0D701CD92DC9260E08C
:105F500070E080E89FEFC111FFC060E070E080E872
:105F60009FE7FAC05801BBCFDB3229F485010E5FF1
:105F70001F4FF501D181C0E0C6CF43E050E068E19A
:105F800071E0C5010E949231892BE9F0F80110E01F
:105F900000E020E030E0A9015F01B0ED8B2E8D0E16
:105FA00089E08815C8F19C2E689491F88C2F887030
:105FB000C2FF16C0811102C00F5F1F4F3196D5017D
:105FC000DC91C92DE9CFE114F10429F00E5F1F4FD8
:105FD000F7011183008360E070E080EC9FE7BCC0B4
:105FE000882311F001501109A5E0B0E00E9416339A
:105FF0009B01AC01220F331F441F551F280D311D7B
:10600000411D511D283999E93907490799E1590777
:10601000A8F2C6609C2ED2CFAEEF8A1206C0C3FD96
:106020003CC09C2E689493F8C9CFDF7DD534A9F588
:1060300080818D3239F4C061DF011296818162E086
:1060400070E006C0DF018B32C1F3119661E070E0B1
:1060500080535D01A61AB70A8A30F8F4E0E8CE163C
:10606000ECE0DE065CF4B601660F771F660F771F63
:10607000C60ED71ECC0CDD1CC80ED11C5D01FFEF77
:10608000AF1ABF0A8C9180538A30A8F1C4FF03C0B5
:10609000D194C194D1080C0D1D1DC1FF09C0E1149C
:1060A000F10431F081E0A81AB108D701AD92BC9299
:1060B000CA01B9010E94BF31C370C33009F49058BE
:1060C0004B015C0120E030E0A9010E94BA31882335
:1060D00009F440C0CFE4D1E017FF05C01195019548
:1060E0001109C7E3D1E06E01B8E1CB1AD10880E213
:1060F000E82EF12C0FC0D501B1CFFE0125913591CD
:10610000459154910E191F09C501B4010E94203216
:106110004B015C01D501C4010E151F0574F72497CE
:10612000F594E794CC16DD06A9F78A2F880F8B2FFC
:10613000881F8F3F49F020E030E0A901C501B4017C
:106140000E94BA31811106C082E290E090931B0553
:1061500080931A05C501B401CDB7DEB7ECE00C940D
:106160004B33283008F027E03327DA01990F311D2F
:1061700087FD916000966105710539F432602E5FEC
:106180003D9330E32A95E1F708959F3F30F0803842
:106190007105610509F03C5F3C5F3D93913008F06B
:1061A0008068911DDF93CF931F930F93FF92EF921F
:1061B000192F987F9695E92F96959695E90FFF27C9
:1061C000E355FE4F99273327EE24FF24A701E7016B
:1061D00005900894079428F4360FE71EF81E491F0F
:1061E000511D660F771F881F991F0694A1F7059010
:1061F000079428F4E70EF81E491F561FC11D770F9C
:10620000881F991F661F0694A1F70590079428F42C
:10621000F80E491F561FC71FD11D880F991F661FF3
:10622000771F0694A1F70590079420F4490F561F95
:10623000C71FD81F990F661F771F881F0694A9F7DD
:1062400084911095177041F0D695C795579547954D
:10625000F794E7941A95C1F7E3E5F1E06894159097
:10626000159135916591959105907FE27395E118AF
:10627000F10A430B560BC90BD009C0F7E10CF11E14
:10628000431F561FC91FD01D7EF4703311F48A9529
:10629000E6CFE894015030F0080F0AF40027021707
:1062A00008F4202F2395022F7A3328F079E37D9389
:1062B0002A95E9F710C07D932A9589F6069497955B
:1062C0006795379517951794E118F10A430B560B0C
:1062D000C90BD00998F023957E9173957A3308F015
:1062E00070E37C932013B8F77E9170617D9330F05A
:1062F000839571E37D9370E32A95E1F71124EF9084
:10630000FF900F911F91CF91DF91992787FD909575
:10631000089591110C948D32803219F08950855076
:10632000C8F70895FB01DC014150504088F08D9181
:1063300081341CF08B350CF4805E659161341CF067
:106340006B350CF4605E861B611171F3990B089537
:10635000881BFCCFDC01FC01672F71917723E1F7EB
:10636000329704C07C916D9370836291AE17BF0722
:10637000C8F308950E94FC3108F481E00895E89480
:1063800009C097FB3EF490958095709561957F4F7D
:106390008F4F9F4F9923A9F0F92F96E9BB2793952B
:1063A000F695879577956795B795F111F8CFFAF43B
:1063B000BB0F11F460FF1BC06F5F7F4F8F4F9F4F6C
:1063C00016C0882311F096E911C0772321F09EE8CA
:1063D000872F762F05C0662371F096E8862F70E030
:1063E00060E02AF09A95660F771F881FDAF7880F0A
:1063F0009695879597F90895990F0008550FAA0B60
:10640000E0E8FEEF16161706E807F907C0F01216C7
:106410001306E407F50798F0621B730B840B950BCA
:1064200039F40A2661F0232B242B252B21F408951F
:106430000A2609F4A140A6958FEF811D811D0895BC
:106440000E9433320C94A7320E94993238F00E9495
:10645000A03220F0952311F00C9490320C949632D7
:1064600011240C94DB320E94B83270F3959FC1F373
:10647000950F50E0551F629FF001729FBB27F00DF2
:10648000B11D639FAA27F00DB11DAA1F649F662747
:10649000B00DA11D661F829F2227B00DA11D621F96
:1064A000739FB00DA11D621F839FA00D611D221F50
:1064B000749F3327A00D611D231F849F600D211D34
:1064C000822F762F6A2F11249F5750409AF0F1F0B7
:1064D00088234AF0EE0FFF1FBB1F661F771F881F20
:1064E00091505040A9F79E3F510580F00C94903296
:1064F0000C94DB325F3FE4F3983ED4F386957795B6
:106500006795B795F795E7959F5FC1F7FE2B880FC5
:10651000911D9695879597F908959927882708954D
:1065200097F99F6780E870E060E008959FEF80EC46
:10653000089500240A9416161706180609060895E9
:1065400000240A9412161306140605060895092E4F
:106550000394000C11F4882352F0BB0F40F4BF2BBE
:1065600011F460FF04C06F5F7F4F8F4F9F4F0895FE
:1065700057FD9058440F551F59F05F3F71F04795F4
:10658000880F97FB991F61F09F3F79F087950895D9
:10659000121613061406551FF2CF4695F1DF08C0F8
:1065A000161617061806991FF1CF86957105610515
:1065B00008940895E894BB2766277727CB0197F9BD
:1065C0000895F999FECF92BD81BDF89A992780B5BB
:1065D0000895262FF999FECF1FBA92BD81BD20BD27
:1065E0000FB6F894FA9AF99A0FBE01960895052EFF
:1065F00097FB1EF400940E940E3357FD07D00E94B3
:10660000603307FC03D04EF40C940E335095409544
:10661000309521953F4F4F4F5F4F0895909580954E
:10662000709561957F4F8F4F9F4F08950E948233E1
:10663000A59F900DB49F900DA49F800D911D1124D6
:106640000895B7FF0C9416330E941633821B930BE8
:1066500008952F923F924F925F926F927F928F9206
:106660009F92AF92BF92CF92DF92EF92FF920F93E1
:106670001F93CF93DF93CDB7DEB7CA1BDB0B0FB6EB
:10668000F894DEBF0FBECDBF09942A8839884888A8
:106690005F846E847D848C849B84AA84B984C8843E
:1066A000DF80EE80FD800C811B81AA81B981CE0F35
:1066B000D11D0FB6F894DEBF0FBECDBFED0108951A
:1066C000A1E21A2EAA1BBB1BFD010DC0AA1FBB1FF6
:1066D000EE1FFF1FA217B307E407F50720F0A21B68
:1066E000B30BE40BF50B661F771F881F991F1A94D5
:1066F00069F760957095809590959B01AC01BD01FF
:10670000CF010895A29FB001B39FC001A39F700D58
:10671000811D1124911DB29F700D811D1124911DA9
:1067200008955058BB27AA270E94A9330C94A7327A
:106730000E94993238F00E94A03220F039F49F3F35
:1067400019F426F40C9496320EF4E095E7FB0C94C1
:106750009032E92F0E94B83258F3BA1762077307D4
:106760008407950720F079F4A6F50C94DA320EF43C
:10677000E0950B2EBA2FA02D0B01B90190010C0151
:10678000CA01A0011124FF27591B99F0593F50F469
:10679000503E68F11A16F040A22F232F342F4427C1
:1067A000585FF3CF469537952795A795F0405395B9
:1067B000C9F77EF41F16BA0B620B730B840BBAF089
:1067C0009150A1F0FF0FBB1F661F771F881FC2F7F4
:1067D0000EC0BA0F621F731F841F48F48795779508
:1067E0006795B795F7959E3F08F0B0CF9395880FC2
:1067F00008F09927EE0F9795879508950E94993292
:1068000060F080E891E009F49EEF0E94A03228F049
:1068100040E851E071F45EEF0CC00C9496320C9499
:10682000DA32E92FE0780E94B83240F3092E052AC7
:10683000B1F3261737074807590738F00E2E07F827
:10684000E02569F0E025E0640AC0EF6307F80094F2
:1068500007FADB01B9019D01DC01CA01AD01EF932B
:106860000E9487340E94A7320E9441345F915523D1
:1068700039F02BED3FE049E450FD49EC0C949233A4
:106880000895DF93DD27B92FBF7740E85FE3161641
:10689000170648075B0718F4D92F0E9444359F93C9
:1068A0008F937F936F930E94E235E8E6F0E00E94B9
:1068B00018350E94A7322F913F914F915F910E940E
:1068C0003332DD2351F09058A2EA2AED3FE049EC43
:1068D0005FE3D0785D270E94A933DF910C94A73243
:1068E0000E9484340C94A7320E94A03258F00E9477
:1068F000993240F029F45F3F29F00C949032511105
:106900000C94DB320C9496320E94B83268F39923CF
:10691000B1F3552391F3951B550BBB27AA2762179B
:106920007307840738F09F5F5F4F220F331F441FA8
:10693000AA1FA9F335D00E2E3AF0E0E832D09150DC
:106940005040E695001CCAF72BD0FE2F29D0660FC9
:10695000771F881FBB1F261737074807AB07B0E80C
:1069600009F0BB0B802DBF01FF2793585F4F3AF012
:106970009E3F510578F00C9490320C94DB325F3FCF
:10698000E4F3983ED4F3869577956795B795F79598
:106990009F5FC9F7880F911D9695879597F9089580
:1069A000E1E0660F771F881FBB1F6217730784071C
:1069B000BA0720F0621B730B840BBA0BEE1F88F72B
:1069C000E09508950E94E9346894B1110C94DB328B
:1069D00008950E94C03288F09F5798F0B92F9927E8
:1069E000B751B0F0E1F0660F771F881F991F1AF0BA
:1069F000BA95C9F714C0B13091F00E94DA32B1E013
:106A000008950C94DA32672F782F8827B85F39F011
:106A1000B93FCCF3869577956795B395D9F73EF452
:106A200090958095709561957F4F8F4F9F4F0895FA
:106A3000DF93CF931F930F93FF92EF92DF927B012F
:106A40008C01689406C0DA2EEF010E943332FE01F9
:106A5000E894A5912591359145915591A6F3EF01C3
:106A60000E94A933FE019701A801DA9469F7DF902B
:106A7000EF90FF900F911F91CF91DF9108950E94A9
:106A8000FC3108F48FEF08959B01AC0160E070E0E9
:106A900080E89FE30C947034FA01EE0FFF1F3096EC
:106AA00021053105A1F16115710561F48038BFE35D
:106AB0009B0749F168949038810561F08038BFEFF9
:106AC0009B0741F099234AF5FF3FE1053105210578
:106AD00019F1E8940894E795D901AA2329F4AB2F7A
:106AE000BE2FF85FD0F310C0FF5F70F4A695E0F7FB
:106AF000F73950F019F0FF3A38F49F779F930DD093
:106B00000F9007FC9058089546F00C94963260E080
:106B100070E080E89FE308954FE79F775F934F937E
:106B20003F932F930E947C362F913F914F915F911D
:106B30000E9420320C94F33519F416F40C9496321A
:106B40000C9425360E94C032B8F39923C9F3B6F3EA
:106B50009F57550B87FF0E9433360024A0E640EA7A
:106B6000900180585695979528F4805C660F771FA2
:106B7000881F20F026173707480730F4621B730B75
:106B8000840B202931294A2BA69517940794202598
:106B900031254A2758F7660F771F881F20F02617E0
:106BA0003707480730F4620B730B840B200D311D3F
:106BB000411DA09581F7B901842F9158880F9695B2
:106BC000879508959B01AC010C9420320E94FC3102
:106BD000880B990B089529F416F00C9490320C94BC
:106BE000DA320C9496320E94C032A8F39638A0F79D
:106BF00007F80F92E8942BE33AEA48EB5FE70E942C
:106C000036320F920F920F924DB75EB70F920E94DD
:106C1000C436E5E9F0E00E9418354F915F91EF919D
:106C2000FF91E595EE1FFF1F49F0FE57E0684427EE
:106C3000EE0F441FFA95E1F74195550B0E943E3641
:106C40000F9007FE0C94443508959F3F31F091500A
:106C500020F4879577956795B795880F911D969540
:106C6000879597F9089591505040660F771F881FB8
:106C7000D2F708950C9490320C9425360E94C032BD
:106C8000D8F39923C9F3940F511DA3F391505040A9
:106C900094F059F0882332F0660F771F881F9150C7
:106CA0005040C1F79E3F51052CF7880F911D9695D6
:106CB000879597F908955F3FACF0983E9CF0BB270D
:106CC000869577956795B79508F4B1609395C1F768
:106CD000BB0F58F711F460FFE8CF6F5F7F4F8F4F06
:106CE0009F4FE3CF0C94DB3216F00C9425360C94B6
:106CF000963268940C9490320E94C032A8F3992383
:106D0000C1F3AEF3DF93CF931F930F93FF92C92F7D
:106D1000DD2788232AF02197660F771F881FDAF76F
:106D200020E030E040E85FEB9FE3883920F0803ED0
:106D300038F021968F770E949233EDEBF0E004C09B
:106D40000E949233EAEEF0E00E9418358B01BE01FA
:106D5000EC01FB2E6F5771097595771F880B990B06
:106D60000E94C13128E132E741E35FE30E94333200
:106D7000AF2D9801AE01FF900F911F91CF91DF9140
:106D80000E94A9330C94A732FA01DC01AA0FBB1FA1
:106D90009B01AC01BF5728F42227332744275078A2
:106DA00020C0B75190F4AB2F002446953795279516
:106DB000011CA395D2F3002071F0220F331F441F52
:106DC000B395DAF30ED00C94913361307105A0E8DD
:106DD0008A07B94630F49B01AC01662777278827DC
:106DE0009078309621F02083318342835383089535
:106DF000DB018F939F930E941633BF91AF91A29FA7
:106E0000800D911DA39F900DB29F900D11240895A8
:106E1000AA1BBB1B51E107C0AA1FBB1FA617B707C0
:106E200010F0A61BB70B881F991F5A95A9F78095DC
:106E30009095BC01CD01089597FB072E16F40094A0
:106E400007D077FD09D00E94083707FC05D03EF433
:106E5000909581959F4F0895709561957F4F089506
:106E6000EE0FFF1F0590F491E02D09940F931F93EF
:106E7000CF93DF938230910510F482E090E0E091AF
:106E80001E05F0911F0530E020E0B0E0A0E0309753
:106E900099F42115310509F44AC0281B390B243017
:106EA0003105D8F58A819B816115710589F1FB0156
:106EB00093838283FE0111C040815181028113813D
:106EC00048175907E0F04817590799F4109761F0EF
:106ED00012960C93129713961C933296CF01DF9162
:106EE000CF911F910F91089500931E0510931F05D8
:106EF000F4CF2115310551F04217530738F0A9019D
:106F0000DB019A01BD01DF01F801C1CFEF01F9CF2B
:106F100090931F0580931E05CDCFFE01E20FF31F56
:106F2000819391932250310939832883D7CF2091BF
:106F30001C0530911D05232B41F420911A0130913D
:106F40001B0130931D0520931C05209118013091E1
:106F500019012115310541F42DB73EB740911C01AF
:106F600050911D01241B350BE0911C05F0911D056E
:106F7000E217F307A0F42E1B3F0B2817390778F010
:106F8000AC014E5F5F4F2417350748F04E0F5F1F6F
:106F900050931D0540931C05819391939FCFF0E082
:106FA000E0E09CCFCF93DF930097E9F0FC013297AC
:106FB00013821282A0911E05B0911F05ED0130E0F1
:106FC00020E01097A1F420813181820F931F20913E
:106FD0001C0530911D052817390709F061C0F09391
:106FE0001D05E0931C05DF91CF910895EA01CE17AE
:106FF000DF07E8F54A815B819E0141155105B1F734
:10700000E901FB83EA8349915991C40FD51FEC171D
:10701000FD0761F4808191810296840F951FE9013B
:1070200099838883828193819B838A83F0E0E0E067
:1070300012968D919C9113970097B9F52D913C91E3
:107040001197CD010296820F931F20911C0530915C
:107050001D052817390739F6309751F510921F058D
:1070600010921E05B0931D05A0931C05BCCFD383C1
:10707000C28340815181840F951FC817D90761F4DD
:107080004E5F5F4F88819981480F591F518340831C
:107090008A819B81938382832115310509F0B0CFCA
:1070A000F0931F05E0931E059ECFFD01DC01C0CFCC
:1070B00013821282D7CFB0E0A0E0E1E6F8E30C94AF
:1070C0002B338C01009751F4CB010E9436378C0191
:1070D000C801CDB7DEB7E0E10C944733FC01E60F01
:1070E000F71F9C0122503109E217F30708F49DC0F5
:1070F000D901CD91DC911197C617D70798F0C5300B
:10710000D10530F3CE0104978617970708F3C61B05
:10711000D70B2297C193D1936D937C93CF010E949B
:10712000D237D6CF5B01AC1ABD0A4C018C0E9D1E26
:10713000A0911E05B0911F05512C412CF12CE12C82
:10714000109731F580911C0590911D0588159905C2
:1071500009F05CC04616570608F058C08091180127
:1071600090911901009741F48DB79EB740911C0191
:1071700050911D01841B950BE817F90708F055C0C5
:10718000F0931D05E0931C05F90171836083A0CF86
:107190008D919C91119712966C90129713967C90FA
:1071A0001397A815B90559F56C0142E0C40ED11C1E
:1071B000CA14DB0420F1AC014A195B09DA0112960A
:1071C000159780F06282738251834083D9016D9359
:1071D0007C93E114F10471F0D7011396FC93EE93C4
:1071E000129776CF22968C0F9D1FF9019183808391
:1071F000F301EFCFF0931F05E0931E0569CF48160A
:10720000590608F42C017D01D3019ACFCB010E94CD
:1072100036377C01009749F0AE01B8010E94203951
:10722000C8010E94D237870153CF10E000E050CF51
:107230009111089581568A5108F480528558089515
:10724000FB01DC0102C001900D9241505040D8F783
:107250000895FB01DC0101900D920020E1F70895F3
:10726000FB01DC014150504030F08D9101908019BC
:1072700019F40020B9F7881B990B0895FB01DC0174
:107280004150504048F001900D920020C9F701C0D4
:107290001D9241505040E0F70895FB015191552354
:1072A000A9F0BF01DC014D9145174111E1F759F4F7
:1072B000CD010190002049F04D9140154111C9F3D5
:1072C000FB014111EFCF81E090E00197089511E0BB
:1072D000C1EED1E004C0FE010E9430372196C23ECB
:1072E000D107C9F7F894FFCF0000A040C800000004
:1072F00075440080894401160064000000F04101DB
:107300000000200580005E00BC0077010000000046
:10731000FA023F0287024703B8029602AA0200005F
:10732000000064093709A5092709EC060C022809A1
:1073300000000000EB06A80DF3064A10FD0F0D0A31
:1073400000484D433538383300436F6D70617373B7
:107350003A2000286465672920004E20004500532C
:1073600020005700732000296D4700203D3E005645
:10737000657273696F6E3A200023007300534C20CE
:10738000503D00506120697320756E6C696B656CAF
:10739000792100536561206C6576656C20503D0055
:1073A000206850610055565A002C0023496E636FC7
:1073B000727265637421204D533D3132334433443E
:1073C0003500496E636C2E20616E672E2878207917
:1073D000207A292F6465673A20003E6128782C794D
:1073E0002C7A292F673A00613D0020670054003D48
:1073F0004E6F2053656E736F7221005428312C320A
:107400002C33293D00206F4320445320546865727B
:107410006D6F6D6574657200543D006F43200048C8
:107420003D0025006F4320413D006D0023456E6106
:10743000626C65002344697361626C6500444400BA
:10744000414E4D4C3033004E616E6F413267320019
:1074500073657269616C3A20002D35002D34002D62
:027460003300F7
:107E0000112484B714BE81FFF0D085E080938100F7
:107E100082E08093C00088E18093C10086E0809377
:107E2000C20080E18093C4008EE0C9D0259A86E02C
:107E300020E33CEF91E0309385002093840096BBD3
:107E4000B09BFECF1D9AA8958150A9F7CC24DD24C4
:107E500088248394B5E0AB2EA1E19A2EF3E0BF2EE7
:107E6000A2D0813461F49FD0082FAFD0023811F036
:107E7000013811F484E001C083E08DD089C08234E0
:107E800011F484E103C0853419F485E0A6D080C0E4
:107E9000853579F488D0E82EFF2485D0082F10E0AE
:107EA000102F00270E291F29000F111F8ED06801E7
:107EB0006FC0863521F484E090D080E0DECF843638
:107EC00009F040C070D06FD0082F6DD080E0C81688
:107ED00080E7D80618F4F601B7BEE895C0E0D1E017
:107EE00062D089930C17E1F7F0E0CF16F0E7DF06D8
:107EF00018F0F601B7BEE89568D007B600FCFDCFD4
:107F0000A601A0E0B1E02C9130E011968C91119780
:107F100090E0982F8827822B932B1296FA010C0160
:107F200087BEE89511244E5F5F4FF1E0A038BF0790
:107F300051F7F601A7BEE89507B600FCFDCF97BE46
:107F4000E89526C08437B1F42ED02DD0F82E2BD052
:107F50003CD0F601EF2C8F010F5F1F4F84911BD097
:107F6000EA94F801C1F70894C11CD11CFA94CF0C13
:107F7000D11C0EC0853739F428D08EE10CD085E9AC
:107F80000AD08FE07ACF813511F488E018D01DD067
:107F900080E101D065CF982F8091C00085FFFCCF94
:107FA0009093C60008958091C00087FFFCCF809118
:107FB000C00084FD01C0A8958091C6000895E0E648
:107FC000F0E098E1908380830895EDDF803219F02E
:107FD00088E0F5DFFFCF84E1DECF1F93182FE3DFCA
:107FE0001150E9F7F2DF1F91089580E0E8DFEE27F6
:047FF000FF270994CA
:027FFE00040479
:00000001FF
